:020000040800F2
:10000000E813002059020008C92C00085315000805
:10001000B92B000889090008033C00080000000013
:10002000000000000000000000000000893300080C
:100030007D0A000800000000612D0008553A000804
:1000400073020008730200087302000873020008BC
:1000500073020008730200087302000873020008AC
:10006000730200087302000873020008730200089C
:100070007302000873020008E9090008730200080F
:1000800073020008090A00087302000873020008DE
:10009000730200087302000873020008730200086C
:1000A000730200087302000873020008730200085C
:1000B000730200083D3B0008730200087302000849
:1000C000730200087302000873020008730200083C
:1000D00073020008F53B0008F73B0008FB3B0008F3
:1000E000730200087302000873020008730200081C
:1000F000730200087302000873020008730200080C
:1001000073020008730200087302000873020008FB
:10011000730200087302000873020008F13B000834
:10012000290A0008590A000873020008730200082F
:1001300073020008730200087302000873020008CB
:1001400073020008730200087302000873020008BB
:10015000730200085D0A000873020008FF3B0008F4
:10016000730200087302000873020008730200089B
:100170007302000873020008730200080000000008
:10018000730200087302000800F002F800F054F84F
:100190000AA090E8000C82448344AAF10107DA45E2
:1001A00001D100F049F8AFF2090EBAE80F0013F0E0
:1001B000010F18BFFB1A43F0010318470479000030
:1001C000247900000A4410F8014B14F00F0508BF11
:1001D00010F8015B240908BF10F8014B6D1E05D013
:1001E00010F8013B6D1E01F8013BF9D1641E03D0EC
:1001F000641E01F8015BFBD19142E4D3704700001B
:100200000023002400250026103A28BF78C1FBD81F
:10021000520728BF30C148BF0B607047632900F008
:100220003E82732900F04382002070471FB507F01B
:10023000DDFA1FBD10B510BD00F078FA1146FFF7CA
:10024000F5FF05F063FF00F096FA03B4FFF7F2FF45
:1002500003BC00F099FA00000948804709480047AC
:10026000FEE7FEE7FEE7FEE7FEE7FEE7FEE7FEE766
:10027000FEE7FEE704480549054A064B70470000C3
:100280002D3B000889010008E80D0020E81300203C
:10029000E80F0020E80F002053EA020C00F069800C
:1002A0002DE9F04B4FF00006002B1FBFB3FA83F58A
:1002B00003FA05F424FA05F65E4012BF1643B2FABB
:1002C00082F502FA05F4C5F120051EBF22FA05FCED
:1002D00044EA0C04203556EA044C4FEA144418BF93
:1002E000641C4FF000084FF00009904271EB030CC2
:1002F00039D3002919BFB1FA81F701FA07F6B0FA2C
:1003000080F700FA07F6C7F120071EBF20FA07FCA6
:1003100046EA0C062037B6FBF4FCA7EB0507103FB6
:1003200007F01F0BCBF120060CFA0BFB2CFA06F69C
:1003300044BFB3460026202FA4BF5E464FF0000BFB
:100340005BEA060C08BF4FF0010B19EB0B09ABFB86
:10035000027C48EB0608C01B06FB02CC0BFB03CC5F
:1003600071EB0C01C1E70B46024641464846BDE829
:10037000F08B13B54FF000004FF00001AFF3008099
:10038000BDE81C40704700000FB41CB50C0007AA64
:10039000009001D02044401E074B7B4469460190E9
:1003A000069800F052F9002C03D06946002000F0B6
:1003B0005FF91CBC5DF814FBDD0200002DE9F04183
:1003C0000E460446002020622046E168884730B38C
:1003D000252805D0D4E901219047206A401CF2E786
:1003E000E168204600278847050018D0A5F14100A4
:1003F000192802D820354FF4006732462946204696
:100400002760FFF70BFF40B1012804D0F61D26F04E
:1004100007060836D8E7361DD6E72846DAE7206A09
:10042000BDE8F08170B50C460546012A05D0287854
:10043000800600D5EA69002302E0012305E05B1C89
:10044000934202D2E05C0028F9D1A869E618C01AEC
:10045000A861286A184428622846AFF3008004E0A7
:10046000D5E9012114F8010B9047B442F8D328468E
:10047000AFF3008070BD10B5431C02E010F8011B03
:1004800071B18107FAD14FF0013202C88C1A8C4346
:1004900014EAC211F9D0C01A0A0603D0C01E10BD5A
:1004A000C01A10BD0A0401D0801E10BD0902FCD084
:1004B000401E10BD40EA010370B59B072ED14FF0DE
:1004C0000136042A2AD308C810C99D1B9D43121F58
:1004D00015EAC61517D0D8B2E1B2401A50EA056144
:1004E00010D198B2A1B2401A50EA05410AD123F0C6
:1004F0007F4024F07F41401A50EA052102D1180EB6
:10050000A0EB146070BDA342DBD018BA21BA8842B8
:1005100001D9012070BD4FF0FF3070BD0AB9002035
:1005200070BD10F8013B11F8014B63B1A3420AD131
:10053000521E08D010F8013B11F8014B1BB1A34229
:1005400001D1521EEDD1181B70BD032A40F230803C
:1005500010F0030C00F0158011F8013BBCF1020F04
:10056000624498BF11F801CB00F8013B38BF11F885
:10057000013BA2F1040298BF00F801CB38BF00F89C
:10058000013B11F0030300F09680083AC0F00880A8
:1005900051F8043B083A51F804CBA0E80810F5E7FD
:1005A000121D5CBF51F8043B40F8043BAFF30080E0
:1005B000D20724BF11F8013B11F801CB48BF11F855
:1005C000012B24BF00F8013B00F801CB48BF00F825
:1005D000012B70474FF0000200B513469446964633
:1005E000203922BFA0E80C50A0E80C50B1F1200146
:1005F000BFF4F7AF090728BFA0E80C5048BF0CC0F4
:100600005DF804EB890028BF40F8042B08BF704751
:1006100048BF20F8022B11F0804F18BF00F8012BC3
:10062000704770477047704710B500F077F8006862
:1006300010BD10B5044600F071F8046010BD000054
:1006400001694A1C02610878704700B58FB0CDE996
:1006500001310021059105497944CDE90310114686
:100660006846FFF7ABFE0FB000BD0000E5FFFFFFDF
:100670000A6802F8010B0A607047D1E900239A4228
:1006800002D2531C0B601070704710B5436913B150
:10069000AFF3008001E0FFF7C5FE012010BD127826
:1006A00000F124010A7000224A700122EDE711686E
:1006B0004FF0FF32E9E710B5203AC0F00B80B1E807
:1006C0001850203AA0E81850B1E81850A0E8185087
:1006D000BFF4F5AF5FEA027C24BFB1E81850A0E890
:1006E000185044BF18C918C0BDE810405FEA827CAA
:1006F00024BF51F8043B40F8043B08BF7047D207C1
:1007000028BF31F8023B48BF11F8012B28BF20F861
:10071000023B48BF00F8012B7047000000487047BB
:10072000880D002000487047880D00207546FFF7AF
:10073000F9FFAE4605006946534620F0070085469E
:1007400018B020B5FFF796FDBDE820404FF0000639
:100750004FF000074FF000084FF0000B21F00701A9
:10076000AC46ACE8C009ACE8C009ACE8C009ACE8EC
:10077000C0098D46704710B50446AFF3008020468F
:10078000BDE81040FFF761BD01491820ABBEFEE790
:1007900026000200704700002DE9F04107462DEDCC
:1007A000028B82B00025474EDFF81C81474C0DE0DC
:1007B0002168491C21603068814207DB256094ED87
:1007C000040B02B0BDEC028BBDE8F0810121404674
:1007D00001F039F90028EBD1082F2CD2DFE807F01F
:1007E00004090E13181D22270821012000F076F8B5
:1007F00021E01821012000F071F81CE028210120DF
:1008000000F06CF817E03821012000F067F812E0E2
:100810004821012000F062F80DE05821012000F08D
:100820005DF808E06821012000F058F803E0782125
:10083000012000F053F8FC20019001231A4601A981
:10084000234800F0ADFC019501231A4601A9204878
:1008500000F0A6FC0120019001231A4601A91C48C2
:1008600000F09EFC012303226946194800F0ECFBCE
:100870009DF800009DF80110000440EA01209DF859
:10088000021008436060A0609FED128B01020ED53C
:10089000C043C0F31600401C4042A06006F0F9FBC4
:1008A00053EC182B06F0ACFCC4E9040107E006F099
:1008B000F0FB53EC182B06F0A3FCC4E9040194ED03
:1008C000040B7EE718000020000C024038020020D4
:1008D0006803002085F90F270088433F2DE9F34185
:1008E00082B007460025164C164EDFF85C8008E003
:1008F0002168491C21603068814202DB2560BDE827
:10090000FF810121404601F09EF80028F0D107F058
:100910000F0040F05000019001231A4601A90B4836
:1009200000F03EFC019501231A4601A9074800F09A
:1009300037FC01231A4603A9044800F031FCDEE726
:100940003802002018000020000C0240680300203C
:1009500010B502200B49886106210020FFF7BEFF79
:1009600008210120FFF7BAFF00210220FFF7B6FFA0
:10097000F0210320FFF7B2FF0021BDE81040042062
:10098000FFF7ACBF000C0240FEE7000070B5124854
:100990004FF4001253100578104894101049092D97
:1009A00007D2DFE805F0060507090B0E1012140048
:1009B000826170BD836170BD846170BD04218161FD
:1009C00070BD8A6170BD8B6170BD8C6170BD80200F
:1009D0000449886170BD00005C02002000100240E4
:1009E00000040240000C024006480168C1F3C061E7
:1009F000002905D04FF000618160032100F0B0BEF6
:100A0000704700000060024006484168C1F3405151
:100A1000002905D04FF40011C160062100F0A0BEEE
:100A2000704700000060024009480168C1F34011AE
:100A3000002902D0074A012111702021816001683C
:100A4000C1F3C001002901D0082181607047000076
:100A5000006402403C0000207047000006484168E6
:100A6000C1F34051002905D04FF40011C1600621A7
:100A700000F076BE7047000000640240704772B616
:100A8000FEE70000024931F8100080B27047000014
:100A900078010020024931F8100080B27047000050
:100AA000B800002010B51038C21700EB5272084C85
:100AB000D310E35C22F00702821A012404FA02F048
:100AC000184201D00C7010BD0020087010BD00004D
:100AD000140C002010B5084A02EBD002127800F086
:100AE0000704012303FA04F0104201D00B7010BD7B
:100AF0000020087010BD0000AC0000202DE9F0417E
:100B00002A4C002626610221A22002F093F904F16A
:100B10001005274FA878697800EB0120217827F885
:100B2000110026610221A42002F084F9A8786978D6
:100B300000EB0120217807EB4101088226610221A8
:100B4000A62002F077F9A878697800EB01202178D7
:100B500007EB4101088426610221A82002F06AF90E
:100B6000A878697800EB0120217807EB410108861D
:100B700026610221AA2002F05DF9A878697800EBCD
:100B80000120217807EB4101A1F8400026610221F4
:100B9000AC2002F04FF9A878697800EB01202178A9
:100BA00007EB4101A1F85000BDE8F0815C02002094
:100BB000200C00202DE9F84F0022DFF89C914FF027
:100BC000010803274FF00F0C09F1040AA9F1040BE7
:100BD00008FA02F50B682B40AB426ED10C7904F099
:100BE0000304012C01D0022C15D18668540007FAA9
:100BF00004FE26EA0E06D1F80CE00EFA04FE4EEAD8
:100C0000060EC0F808E04468AC430D79C5F3001542
:100C10009540254345600C79E443A40708D0C56896
:100C2000540007FA04F6B5438E68A6402E43C6600A
:100C30000C7904F00304022C11D1D40800EB8406D3
:100C4000356A5407E40E0CFA04FE25EA0E05D1F8C5
:100C500010E00EFA04FE4EEA050EC6F820E0056824
:100C6000540007FA04F6B5430E7906F00306A640D1
:100C70002E4306604C6814F4403F67D0374C25681B
:100C800045F480452560246804F480440094344C85
:100C900022F003052E19D6F8085894074FEA147E5F
:100CA0000CFA0EF4A5432F4CA04201D1002424E0FD
:100CB0002D4CA04202D101241FE047E02B4CA04262
:100CC00001D1022419E02A4CA04201D1032414E0EE
:100CD000284CA04201D104240FE0274CA04201D1AE
:100CE00005240AE0254CA04201D1062405E0244C4D
:100CF000A04201D1072400E0082404FA0EF42C439A
:100D0000C6F80848D9F800409C434D68ED0200D56C
:100D10001C43C9F80040DAF800409C434D68AD021E
:100D200000D51C43CAF80040DBF800409C434D68E6
:100D3000AD0300D51C43CBF80040074D083D2C689F
:100D40009C434E68F60300D51C432C60521C102AAD
:100D5000FFF43EAFBDE8F88F083C01404438024044
:100D60000030014000000240000402400008024040
:100D7000000C024000100240001402400018024023
:100D8000001C024001488068704700009C00002061
:100D90000248816802781144816070479C000020FD
:100DA00010B50B48016841F400710160016841F41D
:100DB00080610160016841F480710160032000F0EE
:100DC00065F8002000F006F800F026F8002010BDBD
:100DD000003C024070B504460D4D4FF47A712878FE
:100DE000B1FBF0F00B490968B1FBF0F000F09DFB9E
:100DF00008B1012070BD102C07D200222146501EE0
:100E000000F024F86C60002070BD012070BD00006F
:100E10009C000020A800002082B00B48016841F42B
:100E200080410160006800F4804001900648001F86
:100E3000016841F080510160006800F0805001902D
:100E4000052002B000F022B844380240F0B40D464C
:100E50000D4B1B68C3F30223C3F10704042C00D914
:100E60000424191D072901D2002300E0DB1E0126FE
:100E700006FA04F1491E294099409E40761E16400C
:100E80003143F0BC03F026B90CED00E000F007019F
:100E9000054A10684FF6FF03184040EA0120034955
:100EA00008431060704700000CED00E00000FA05F8
:100EB00070B50446002C09D0606A002540B1256158
:100EC0006561A56294F8510040B10CE0012070BD4D
:100ED0006068B0F5827FF4D0E561F2E784F85050A5
:100EE000204600F045F8022084F85100206801688F
:100EF00021F040010160A088218900F4827001F492
:100F000004410843A18901F400610843217C01F0F8
:100F100002010843217D01F001010843218B01F406
:100F200000710843217F01F03801084394F8201034
:100F300001F080010843218D01F40051084321682C
:100F40000860A069042101EA104094F8241001F01F
:100F500010010843216848602068C16921F40061DC
:100F6000C1616565012084F85100002070BD00005A
:100F7000F0B587B00446142102A8FFF72BFB2D4BD8
:100F8000226800242C49022503262C489A421DD1B0
:100F9000294A1432136843F480531360126802F430
:100FA000805201920A6842F001020A60096801F069
:100FB00001010191E0210291039504940596052118
:100FC000069102A9FFF7F6FD07B0F0BD1C4B9A424F
:100FD000FAD1194A1032136843F4004313601268BF
:100FE00002F4004201920A6842F001020A600A68B3
:100FF00002F0010201920A6842F004020A600968E4
:1010000001F0040101914FF4004102910395049411
:1010100005960627069702A9FFF7CCFD4FF4E0508E
:101020000290039504940596069702A90548FFF7D8
:10103000C1FDC9E7003001403038024000000240E5
:10104000003C0040000802402DE9F84F04468A4663
:1010500091461D46002694F85100012801D0022631
:1010600099E060684FF0040BB0F5827F01D1A06871
:1010700020B394F8500001282BD04FF0010884F8D9
:101080005080FFF77FFE0746BAF1000F23D0B9F179
:10109000000F20D084F851B000206065C4F838A05B
:1010A000A4F83C90A4F83E902063A086E0862064DB
:1010B0006064A068B0F5004F0FD018E084F851B01C
:1010C0004B46524651462046009500F033F9BDE8A4
:1010D000F88F0220FBE701265DE02068016821F01F
:1010E000400101602068016821F4804101602068AE
:1010F0000168490603D4016841F040010160E068DD
:10110000B0B133E020688168C90709D0007BA16BCA
:101110000870A06B401CA063E08F401EE08707E0D2
:10112000FFF730FEC01BA84201D3681C04D11DB1DB
:10113000E08F0028E6D11CE0032684F851802AE0E5
:1011400020688168C90709D0C068A16B0880A06BBE
:10115000801CA063E08F401EE08707E0FFF712FECF
:10116000C01BA84201D3681C0FD175B1E08F0028C5
:10117000E6D13A462946204602F023F808B120205D
:101180006065606D28B1012605E0032684F8518072
:1011900001E084F85180002084F85000304696E742
:1011A0002DE9F84F04468B4692461D46002694F8DA
:1011B000500001280DD04FF0010884F85080FFF74F
:1011C000E1FD074694F85100B146012804D00226FB
:1011D000ACE00220BDE8F88FBBF1000F1CD05FEA45
:1011E0000A0019D0032084F85100C4F85490C4F8C0
:1011F00030B0A4F834A0A4F836A0C4F83890A4F80D
:101200003C90A4F83E90C4F84490C4F84090A06884
:10121000B0F5004F02D00BE0012687E0206801689E
:1012200021F0400101602068016841F480410160C3
:1012300020680168490603D4016841F0400101605B
:10124000E068B0F5006F05D0606888B3BAF1010FAF
:101250002FD04FE0606810B1BAF1010F20D1206BA0
:1012600021680088C860206B801C2063E08E401ECF
:10127000E08615E020688168890709D5216B098817
:10128000C160206B801C2063E08E401EE08607E07A
:10129000FFF778FDC01BA84201D3681C04D11DB123
:1012A000E08E0028E6D128E0032684F851803DE056
:1012B000FFE7206B216800780873206B401C2063D7
:1012C000E08E401EE08615E020688168890709D518
:1012D000216B09780173206B401C2063E08E401E57
:1012E000E08607E0FFF74EFDC01BA84201D3681C53
:1012F0000ED16DB1E08E0028E6D13A46294620464F
:1013000001F0A6FF08B120206065A06820B107E0C9
:10131000032684F8518009E02068C1688068009045
:10132000606D08B1012601E084F8518084F8509086
:1013300030464FE72DE9FF4F81B004460E9E8B46A5
:1013400098460125002794F8500001280ED0AA469F
:1013500084F850A0FFF716FD814694F851006168AB
:1013600001280DD0B1F5827F08D103E0022005B03D
:10137000BDE8F08FA16809B9042801D00227CFE0A9
:10138000BBF1000F2DD0039858B35FEA080028D0B6
:1013900094F85100042802D0052084F85100002060
:1013A00060650399A163A4F83E80A4F83C80C4F86A
:1013B00030B0A4F83680A4F83480206460642068DB
:1013C0000168490603D4016841F040010160E0680A
:1013D000B0F5006F07D06068F0B3B8F1010F49D0E5
:1013E0007EE001279CE0606810B1B8F1010F3AD1AE
:1013F000206B21680088C860206B801C2063E08E11
:10140000401EE0862FE02068816889070DD5E18EB7
:1014100059B1012D09D1216B0988C160206B801C55
:101420002063E08E401EE086002520688168C907A1
:101430000BD0E18F49B1C068A16B0880A06B801C04
:10144000A063E08F401EE0870125FFF79BFCA0EB27
:101450000900B04207D300E00CE0701C03D0032762
:1014600084F851A05CE0E08E0028CCD1E08F002809
:10147000C9D13BE0206B216800780873206B401CC9
:101480002063E08E401EE0862AE02068816889079C
:101490000DD5E18E59B1012D09D1216B0978017368
:1014A000206B401C2063E08E401EE08600252068F3
:1014B0008168C9070BD0E18F49B1C068A16B087082
:1014C000A06B401CA063E08F401EE0870125FFF762
:1014D00059FCA0EB0900B04201D3701C10D17EB1C1
:1014E000E08E0028D1D1E08F0028CED14A46314687
:1014F000204601F0ADFE38B10127202060650FE0E5
:10150000032784F851A00BE0A06818B92068C168CF
:1015100080680090606D08B1012701E084F851A057
:10152000002084F85000384621E710B5401EB0F185
:10153000807F01D3012010BD4FF0E02460610F21B6
:10154000601702F0C7FD0020A06107202061002085
:1015500010BDFEE730B500224B68124CA468C4F3FE
:101560000004114DAD68C5F300052C430F4DAD6867
:10157000C5F300052C4302D00122104630BD0C4DAE
:1015800053B10C681C43D1E902310B4341681C4341
:1015900029400C434460F0E7436809682B400B4343
:1015A0004360EAE7002001400021014000220140A1
:1015B000E010FCFF30B500228368C3F30003002B6A
:1015C00002D00122104630BD8C680B68234344686A
:1015D000054D2C40234343608368496823F400632E
:1015E0000B438360EEE70000FFFEFFFC30B50022F6
:1015F0004B688468C4F30004002C02D0012210461A
:1016000030BD33B143688C6823F46843234343609F
:1016100003E0436823F468434360D1E90334234380
:101620008468074D2C400D6805F070652C432343FA
:1016300083604968C36A23F470030B43C362DEE727
:10164000FDFCFFC010B54FF4407494FAA4F401F40B
:101650004073B4FA84F4E34000EB8300C36A01F002
:101660001F011F248C4002F01F02A3438A40134332
:10167000C36210BD70B54FF0007494FAA4F401F089
:101680000073B4FA84F4E34000EB8300C4684FF0C5
:10169000F87393FAA3F501F0F871B5FA85F521FA1C
:1016A00005F50726AE4093FAA3F3B3FA83F3D940C6
:1016B000B4438A401443C46070BD000008B50449B7
:1016C0000A6802430A6009680140009108BD0000F1
:1016D0003038024008B504490A6802430A600968C4
:1016E0000140009108BD00003038024008B50449AF
:1016F0000A6802430A6009680140009108BD0000C1
:101700003038024008B504490A6802430A60096893
:101710000140009108BD00004038024008B504496E
:101720000A6802430A6009680140009108BD000090
:101730004038024008B504490A6802430A60096853
:101740000140009108BD000044380240034A1430B3
:10175000515C0A5822F004020A507047CF79000801
:10176000034A515C425822F0010242507047000087
:10177000C7790008034A515C425842F010024250B7
:1017800070470000CF790008034A515C425842F08C
:101790000102425070470000CF790008034B595CAA
:1017A000435823F06063134343507047CF790008D8
:1017B000044B001D595C0B586FF30F0313430B5080
:1017C00070470000CF790008034B595C435823F061
:1017D000C003134343507047CF790008034B595C53
:1017E000435823F48063134343507047CF79000874
:1017F000034B595C435823F4C04313434350704791
:10180000CF790008034B595C435823F4907313437A
:1018100043507047CF790008034B595C435823F479
:101820000073134343507047CF790008034B595C52
:10183000435823F4C053134343507047CF790008F3
:10184000034B595C435823F44033134343507047D0
:10185000CF79000830B500222B4C0379251F016891
:10186000002B47D099B343798BB1012B17D0022BB2
:101870001DD00122817951B3234C0834231F012943
:101880001DD0022924D003292BD0012239E023685E
:101890008B43236001682B680B432B60EAE72B68BE
:1018A0008B432B60016823680B432360E2E72B68BE
:1018B0000B432B60016823680B432360DAE7016860
:1018C00025688D432560006819680143196018E098
:1018D00001681D688D431D60006821680143216017
:1018E0000FE001681D680D431D6000682168014319
:1018F000216006E02B688B432B60006821688143E0
:101900002160104630BD0000043C01402DE9F0414B
:101910000A6892FAA2F2B2FA82F30F2603258AE04D
:1019200001249C402240002A7DD04C68012C01D02B
:10193000022C1BD18C68876892FAA2FCBCFA8CFC42
:101940004FEA4C0C05FA0CFC27EA0C0792FAA2FCB1
:10195000BCFA8CFC4FEA4C0C04FA0CF42743876069
:10196000CC68476854439743274347600C69C7686E
:1019700092FAA2FCBCFA8CFC4FEA4C0C05FA0CFC67
:1019800027EA0C0792FAA2FCBCFA8CFC4FEA4C0C3A
:1019900004FA0CF42743C7604C68022C34D192FA45
:1019A000A2F4B4FA84F4082C16D24C69076A92FAAD
:1019B000A2FCBCFA8CFC4FEA8C0C06FA0CFC27EA61
:1019C0000C0792FAA2FCBCFA8CFC4FEA8C0C04FACD
:1019D0000CF42743076217E04F69D0F824C0140ABB
:1019E00094FAA4F8B8FA88F84FEA880806FA08F8D2
:1019F00094FAA4F4B4FA84F4A4002CEA080CA740E6
:101A00004CEA070CC0F824C04C68076892FAA2FCA4
:101A1000BCFA8CFC4FEA4C0805FA08FC27EA0C07D4
:101A200092FAA2F200E005E0B2FA82F2520094408B
:101A3000274307605B1C0A6832FA03F47FF470AF37
:101A40000020BDE8F0810069814301D0002070478B
:101A5000012070470069814301D0002070470120B8
:101A6000704710B5044601F0A7F9206001F07AF93B
:101A7000606001F085F9A060606801F08FF9E060B6
:101A800010BD10B501220368C3F38013002B25D1CC
:101A9000D1E900231A43D1E9023423431A430B69E5
:101AA0001A434B691A438B691A43CB691A430B6A71
:101AB0001A4303684FF6BF74A3431A430260426897
:101AC0004B6922F0040242EA134242600A6AB2F50C
:101AD000005F02D1898C89B201610022C16921F4C1
:101AE0000061C161104610BD0149086070470000E7
:101AF000A800002010B501291CD004291CD01029F1
:101B00001CD040291CD0B1F5807F1BD0B1F5806F6F
:101B10001AD006210D4B18305B5C184403680B4C3F
:101B2000E41D615C03248C40120CA3438A401343E0
:101B3000036010BD0021EDE70121EBE70221E9E799
:101B40000321E7E70421E5E70521E3E7B27900088F
:101B500010B501291CD004291CD010291CD0402903
:101B60001CD0B1F5807F1BD0B1F5806F1AD0062153
:101B70000D4B18305B5C184403680B4CE41D615C32
:101B8000F0248C40120CA3438A401343036010BD21
:101B90000021EDE70121EBE70221E9E70321E7E777
:101BA0000421E5E70521E3E7B279000810B5012932
:101BB00016D0042916D0102916D0402916D0B1F518
:101BC000807F15D0B1F5806F14D00621036A0A4CCE
:101BD000615C0A248C40A3438A401343036210BD16
:101BE0000021F3E70121F1E70221EFE70321EDE70F
:101BF0000421EBE70521E9E7C079000810B50129C8
:101C00001CD004291CD010291CD040291CD0B1F5AF
:101C1000807F1BD0B1F5806F1AD006210D4B183094
:101C20005B5C184403680B4CE41D615C0C248C4025
:101C3000120CA3438A401343036010BD0021EDE75B
:101C40000121EBE70221E9E70321E7E70421E5E7CA
:101C50000521E3E7B27900082DE9F0410268264C3E
:101C6000264D274E274F284B4FF0804CA04209D0DD
:101C7000604507D0A84205D0B04203D0B84201D099
:101C8000984205D1D1F8048022F0700242EA08029D
:101C9000A0421BD0604519D0A84217D0B04215D041
:101CA000B84213D0984211D0184DA8420ED0184D0A
:101CB000A8420BD0174DA84208D0174DA84205D016
:101CC000164DA84202D0164DA84203D1CD6822F489
:101CD00040722A4302608A68C2620A888262A04215
:101CE00001D0984201D109690163416941F00101C4
:101CF00041610020BDE8F081000001400004004087
:101D000000080040000C0040000401400040014079
:101D1000004401400048014000180040001C004001
:101D200000200040016921F490410161416921F0E6
:101D30002A0141617047143050E8001F41F08001D2
:101D400040E80012002AF7D170470C3050E8001F1D
:101D500041F0200140E80012002AF7D1704700004E
:101D60002DE9FF4104460D4601270026E068C0F337
:101D70004030002841D1E9686868AA6908432969A8
:101D800011430843E16849F20C6291430843E06063
:101D9000A868216921F440510143216168696169A2
:101DA00021F44071014361616846FFF75AFE15480E
:101DB000844201D1039E17E01348844201D1029E60
:101DC00012E01248844201D1029E0DE01048844284
:101DD00001D1039E08E00F48844201D1029E03E036
:101DE0000D48844200D1029E3EB12B682BB10027E2
:101DF00031462046AA6900F011F804B03846BDE823
:101E0000F081000000100140004400400048004004
:101E100000140140004C0040005000402DE9F0410A
:101E200004461927A1FB0778002064253226B2F565
:101E3000004F2BD09C469B0F4FEA8C023846414600
:101E4000FEF72AFA0146B0FBF5F06FF01802504396
:101E500001EB800006EB0010B0FBF5F000F0F002A3
:101E6000B1FBF5F002EB0012B1FBF5F06FF01803D7
:101E7000584301EB800006EB0010B0FBF5F000F0DA
:101E80000F00104480B2A060BDE8F081DA1840EB8A
:101E9000000338464146FEF7FFF90146B0FBF5F076
:101EA0000201B1FBF5F06FF01803584301EB80001D
:101EB00006EBC000B0FBF5F000F0F80002EB4002CA
:101EC000B1FBF5F0584301EB800006EBC000B0FB1E
:101ED000F5F000F00700104480B2A060D4E708B528
:101EE0004FF0E0210A690092421C05D0401C03E03B
:101EF0000A69D20300D5401E0028F9D108BD0000B0
:101F000010B5B2B001228DF8002040F080008DF8AD
:101F1000010003208DF802100146684600F04DFED6
:101F20008DF80300010A05208DF80410084C228A60
:101F3000052A00D3024662826946E068FEF705FB87
:101F4000628A0448E16804F0A9FB32B010BD0000C9
:101F5000000C00200048004010B512494FF48000EA
:101F6000886101F013FA104C012020700A2003F060
:101F7000EDFE01F01DF9FEF7C1FD022020700A20E0
:101F800003F0E4FE01F014F9FEF7B8FD0320207021
:101F90000A2003F0DBFE01F00BF9BDE81040FEF76C
:101FA000ADBD0000001002405C02002030B593B0CF
:101FB000002410941194129414210BA8FEF70AFB2C
:101FC0000794089409940A94182101A8FEF702FBCB
:101FD0004FF480755148016841F4807101600068D8
:101FE00000F4807000904D481438016841F0010100
:101FF0000160006800F001000090072001900320BC
:102000000290059401A94648FFF780FC45494648DF
:1020100002788A58037822F06062CA5002788A589F
:10202000037822F0C002CA5002788A58037822F45A
:102030004032CA5002788A58037822F4907242F4EF
:102040008072CA5002788A58037822F40072CA500B
:1020500002788A58037842F48062CA5002788A581B
:10206000037822F4C05242F40062CA5002788A58BF
:10207000037822F4C04242F40052CA50294902783F
:1020800014315258007822F00402425010941194F6
:102090001295264D10A92846FFF78CFA0B944FF4A1
:1020A00000100C900D940E944FF440700F900BA9FB
:1020B0002846FFF79BFAA86820F48060A8604FF4D8
:1020C00080300790089407A91948FFF743FA4FF0AA
:1020D0000074224621142846FFF7B4FA072221464D
:1020E0002846FFF7C7FA134C40F20521224628463E
:1020F000FFF7A8FA072221462846FFF7BBFA0E4C45
:1021000040F20A2122462846FFF79CFA0722214680
:102110002846FFF7AFFA13B030BD00004438024044
:102120000000024000640240AA790008002001403B
:1021300000230140010030020200600210B54FF49C
:102140008000FFF7C7FA4FF40010FFF7C3FA01F061
:1021500081FF0122002100F0B8FD01460E2001F0B0
:1021600089FF0E2001F04EFF01F074FF01220221D1
:1021700000F0ABFD0146112001F07CFF112001F0C1
:1021800041FF01F067FF0122022100F09EFD0146A0
:10219000382001F06FFF382001F034FF01F05AFFC2
:1021A0000122022100F091FD0146392001F062FF79
:1021B000392001F027FF01F04DFF0122022100F03C
:1021C00084FD0146452001F055FFBDE81040452043
:1021D00001F018BF2DE9F04F89B00024079408944E
:1021E000182101A8FEF7F6F91020FFF767FA04207E
:1021F000FFF764FA8020FFF761FA0120FFF75EFA2B
:102200000220FFF75BFA0820FFF758FADFF8E881B1
:102210007848C8F818004FF47860C8F81800DFF85C
:10222000E0917648C9F81800DFF8D8A14FF08C701B
:10223000CAF81800DFF8D4B17348CBF81800754F0E
:102240007348B8613C2001900125029503940494E1
:10225000059501A94046FFF759FB4FF6C070019064
:10226000029503940494059401A94046FFF74EFBA0
:102270004EF23E000190029503940494059401A946
:102280004846FFF743FB01950294059401A948468F
:10229000FFF73CFB182001900295039404940594E9
:1022A00001A95046FFF732FB40F607400190029526
:1022B00003940494059401A95846FFF727FBA8024C
:1022C000019003260296059401A93846FFF71EFBEC
:1022D0004FF462500190029503940494059501A96E
:1022E0003846FFF713FB4CF2160001900295039459
:1022F0000494059401A93846FFF708FB30020190C9
:10230000029503940494059501A94846FFF7FEFA47
:1023100028020190029503940494059501A9504662
:10232000FFF7F4FAF00201900296059401A95046D5
:10233000FFF7ECFA01950294059501A93846FFF7DD
:10234000E5FA38200190029503940494059501A9BB
:102350005846FFF7DBFA680201900296059401A93E
:102360005846FFF7D3FA01960296059401A9404614
:10237000FFF7CCFA284801684FF4704292FAA2F2B3
:10238000B2FA82F221F4704106FA02F211430160BE
:102390004FF00808CDF81C808DF820508DF82140B2
:1023A0008DF8225007A8FFF755FAF86898FAA8F1B7
:1023B000B1FA81F1490006FA01F1884398FAA8F1CF
:1023C000B1FA81F1490004FA01F10843F860386874
:1023D00098FAA8F1B1FA81F149008E4098FAA8F173
:1023E000B1FA81F14900B0438C402043386009B014
:1023F000BDE8F08F00007CF00010024000003EE3DA
:10240000000802400000024000003F0C00040240AF
:10241000000096F8000C0240083801400C480B49B7
:1024200001604FF48271416000218160C1600161EF
:1024300041614FF4007282611822C26101624162FF
:1024400081620A21C162FEF733BD00000030014005
:102450001003002010B592B0282108A8FEF7BAF8A2
:10246000182102A8FEF7B6F81E48016841F4804121
:102470000160006800F4804001901A48103801683B
:1024800041F002010160006800F0020001904FF489
:1024900070400290022003900320049000240594D1
:1024A00006940520079002A90F48FFF72FFA089419
:1024B0004FF4827009900A940B940C944FF480208E
:1024C0000D900E940F9410940A201190074C08A9B7
:1024D0002046FFF7D6FA616821F01001616012B062
:1024E00010BD0000403802400004024000380040A7
:1024F00010B511480F4901604FF48271416000210D
:102500008160C160016101224261920482613822CE
:10251000C2610162416281620A21C162FEF7C8FCA8
:102520000548FEF7C5FC002803D0BDE81040FEF7C3
:10253000A6BA10BD003C00406803002010B586B06C
:10254000142101A8FEF746F80220FFF7DBF818482F
:102550000068C0F302200122022100F0CFFB0146F7
:102560001D2001F097FD1D2001F059FD5320ADF80D
:1025700004000020029040F2E731039104900D4CDA
:1025800001A92046FFF768FB206840F0800020602A
:10259000A06844F207018843A060606820F07000E2
:1025A0006060A06820F08000A06006B010BD000050
:1025B0000CED00E00004004070B58CB0142107A8B9
:1025C000FEF708F8182101A8FEF704F80420FFF729
:1025D00099F83148016841F002010160006800F09B
:1025E00002000090C0200190022002900024039479
:1025F00004940594069001A92848FFF787F9012063
:10260000ADF81C0008944FF6FF7009900A94244C12
:1026100007A92046FFF720FB206820F080002060FB
:10262000A06820F0070040F00300A060A5132A4630
:1026300001212046FFF75EFA002201212046FFF724
:10264000DDFA4FF44016324601212046FFF780FAAA
:10265000002201212046FFF7A9FA2A461021204630
:10266000FFF748FA002210212046FFF7C7FA32464A
:1026700010212046FFF76CFA002210212046FFF7B8
:1026800095FA606820F070006060A06820F080001B
:10269000A0600CB070BD0000303802400004024061
:1026A0000008004010B586B0142101A8FDF792FF84
:1026B0002020FFF727F815480068C0F30220002209
:1026C000114600F01BFB0146372001F0E3FC3720E8
:1026D00001F0A5FC44F29F10ADF804000020029028
:1026E000132003900A4C01A92046FFF7B5FA206891
:1026F00040F080002060606820F070006060A0689A
:1027000020F08000A06006B010BD00000CED00E0DD
:10271000001400402DE9F0418EB01C2107A8FDF700
:1027200059FF182101A8FDF755FF1020FFF702F807
:102730000120FEF7DBFF4FF40070019002250295A7
:102740000327039700240494059407260696DFF8D0
:10275000708001A94046FFF7D9F868020190029500
:102760000397049401200590069601A94046FFF7BF
:10277000CDF801F077FC0122022100F0D8FA0146E1
:10278000252001F097FC252001F056FC4FF4E130A4
:102790000790089409940A940C200B900C940D94C3
:1027A000084C07A92046FFF7DBFA2046FFF7BAFAE4
:1027B000E16841F40051E1600EB0BDE8F081000035
:1027C00000000240001001402DE9F0418EB01C21B4
:1027D00007A8FDF7FFFE182101A8FDF7FBFE4FF447
:1027E0000030FEF79BFF0820FEF780FF20200190BD
:1027F00002250295032703970024049405940726D5
:102800000696DFF8CC8001A94046FFF77FF840200C
:10281000019002950397049401200590069601A962
:102820004046FFF773F8AA062A4D06212846FEF710
:10283000B5FF402206212846FEF7C6FF00220621EA
:102840002846FEF7FDFFAA1506212846FEF7DAFF07
:10285000002206212846FEF7DFFF2A15062128461A
:10286000FEF7BCFF002206212846FEF7DFFF00220C
:1028700006212846FEF7BCFF06212846FEF766FF24
:1028800001F0F0FB0122022100F051FA014626205E
:1028900001F010FC262001F0CFFB4FF4164007900A
:1028A000089409940A940C200B900C940D940A4CF3
:1028B00007A92046FFF754FA2046FFF733FAE168EC
:1028C00041F40051E16004F0EDF80EB0BDE8F08194
:1028D000000C024000600240004400402DE9F0413D
:1028E0008EB01C2107A8FDF775FE182101A8FDF781
:1028F00071FE4FF48020FEF711FF0820FEF7F6FE70
:102900004FF480700190022502950326039600245F
:102910000494059407270697DFF8E08001A9404654
:10292000FEF7F4FF2802019002950396049401201B
:102930000590069701A94046FEF7E8FFAA06304D2C
:1029400003212846FEF72AFF402203212846FEF7EE
:102950003BFF002203212846FEF772FF00220321DD
:102960002846FEF74FFF002203212846FEF754FFBA
:102970002A1503212846FEF731FF002203212846AD
:10298000FEF754FF002203212846FEF731FF032102
:102990002846FEF7DBFE01F065FB0122002100F076
:1029A000C6F90146272001F085FB272001F044FBF2
:1029B0004FF4E1300790089409940A940C200B908E
:1029C0000C940D940F4C07A92046FFF7C9F9204637
:1029D000FFF7A8F9E06840F40050E060201D0A49C4
:1029E000074AC978083288502046FFF7A4F9032126
:1029F0002846FEF7BFFE0EB0BDE8F081000C024095
:102A00000060024000480040CF7900082DE9F04105
:102A10008EB01C2107A8FDF7DDFD182101A8FDF7E8
:102A2000D9FD2020FEF786FE0420FEF75FFE402041
:102A30000190022502950326039600240494059430
:102A400008270697DFF8608101A94046FEF75EFF80
:102A5000802001900295039604940120059006972A
:102A600001A94046FEF752FF504D4FF02066324616
:102A700001212846FEF792FE002201212846FEF79A
:102A8000A3FE002201212846FEF7DAFEAF153A46E2
:102A900001212846FEF7B6FE002201212846FEF756
:102AA000BBFE4FF48068424601212846FEF796FEA1
:102AB000002201212846FEF7B9FE00220121284606
:102AC000FEF796FE01212846FEF740FE324606211B
:102AD0002846FEF763FE402206212846FEF774FED4
:102AE000002206212846FEF7ABFE3A46062128467C
:102AF000FEF788FE002206212846FEF78DFE42469C
:102B000006212846FEF76AFE002206212846FEF727
:102B10008DFE002206212846FEF76AFE0621284681
:102B2000FEF714FE01F09EFA0122022100F0FFF8E8
:102B30000146472001F0BEFA472001F07DFA4FF42C
:102B400016500790089409940A940C200B900C944A
:102B50000D94174E07A93046FFF702F93046FFF7EC
:102B6000E1F8F06840F40050F06006F10C0454E81D
:102B7000000F40F0100044E800010029F7D10C4894
:102B8000001D0C49094A8979083288503046FFF700
:102B9000D2F806212846FEF7EDFD3046FFF7D5F8BE
:102BA0000EB0BDE8F0810000000802400064024061
:102BB00000140140CF790008FEE730B503464FF618
:102BC000FF70002B15D0814213D04AF201040DE0B2
:102BD00013F8012B50400022C50702D04008604086
:102BE00000E04008521CD2B2082AF5D3491E89B22F
:102BF000EED230BD30B4002848D0022946D3037845
:102C000042781446012B01D0002B3FD1891E052AA2
:102C100037D008DC012A11D0022A14D0032A17D099
:102C2000042A06D119E0062A1CD00F2A1FD0102A28
:102C300022D0204630BC0121FFF762B930BC89B2F6
:102C4000801C00F019B930BC89B2801C00F08CB92E
:102C500030BC89B2801C00F0FBB930BC89B2801C4A
:102C600000F04EBA30BC89B2801C01F031B930BCE2
:102C700089B2801C00F0ECBF30BC89B2801C01F02E
:102C800067B830BC89B2801C01F0DEB830BC704738
:102C900070B50C4D2868E988022911D3421812F842
:102CA000023D527843EA0224891E89B2FFF785FF6C
:102CB000844205D1E9882868BDE87040FFF79ABFD3
:102CC00070BD0000000C0020FEE730B500F00703E7
:102CD000C3F10704042C00D90424181D072801D2CD
:102CE000002300E0DB1E012505FA04F0401E084029
:102CF00098409D406D1E1540284330BD30B500F012
:102D00000703C3F10704042C00D90424181D072865
:102D100001D2002300E0DB1E012505FA04F0401E6D
:102D2000084098409D406D1E1540284330BD30B589
:102D300000F00703C3F10704042C00D90424181D74
:102D4000072801D2002300E0DB1E012505FA04F06C
:102D5000401E084098409D406D1E1540284330BDE0
:102D6000704700000449096801F0F001034A0909AD
:102D7000515CC8407047000008380240D77900080D
:102D80000449096801F4E051034A02EB91210978F2
:102D9000C840704708380240E779000804490968CC
:102DA00001F46041034A02EB51310978C840704791
:102DB00008380240E77900080748006800F00C0175
:102DC0000648002907D0042904D0082903D1082087
:102DD00000F008B802487047083802400024F400A8
:102DE00000127A0010B504460020104B196801F457
:102DF00080020F49002A03D0B2F5800F00D149109C
:102E0000082C11D1186800F03F00B1FBF0F01968F0
:102E1000C1F388114843196801F44031012202EBE3
:102E200011414900B0FBF1F010BD00000438024030
:102E30000024F40038B50C460D4A0023D3600C3250
:102E40001070FDF7A3FD0A2002F080FF084A012060
:102E500010320090631C111F0648FEF76BFA18B180
:102E600000F094FA012038BD00F090FA002038BD3F
:102E70005C020020100300202DE9F04FB3B004469F
:102E80004FF0000AC8216846FDF7A4FB607821785E
:102E900040EA0129E078A17840EA0127B9F15F0F03
:102EA00059D807EB0900602855D8F81DC0F3C70BA7
:102EB00001208DF800008DF8010003248DF802B088
:102EC00000264FF0000825E000210DF80410002531
:102ED00009EB060080B232A9FDF7E4FD9DF8C810A9
:102EE0001DF80400A94008430DF80400761CB6B292
:102EF000BE4202D34FF0010A03E06D1CEDB2082D73
:102F0000E6D3641CE4B2BAF1010F05D008F1010860
:102F100008F0FF08D845D7D321466846FFF74DFE95
:102F2000611CC9B26B460DF80400040A481CC2B209
:102F30005C540B4C208A904200D202466282694661
:102F4000E068FDF702FB628A0648E16803F0A6FB31
:102F500033B0BDE8F08F02210120FEF7D1FFF7E783
:102F6000000C0020004800402DE9F04FB3B04FF0B6
:102F7000000A4178027841EA0229C178807841EA62
:102F80000027B9F15F0F5AD807EB0900602856D81F
:102F9000F81DC0F3C70B01208DF8000002208DF84A
:102FA000010003248DF802B000264FF0000825E050
:102FB00000210DF80410002509EB060080B232A9AB
:102FC000FDF788FD9DF8C8101DF80400A9400843CE
:102FD0000DF80400761CB6B2BE4202D34FF0010ACF
:102FE00003E06D1CEDB2082DE6D3641CE4B2BAF127
:102FF000010F05D008F1010808F0FF08D845D7D324
:1030000021466846FFF7D9FD611CC9B26B460DF831
:103010000400040A481CC2B25C540B4C208A904243
:1030200000D2024662826946E068FDF78EFA628A43
:103030000648E16803F032FB33B0BDE8F08F0221AF
:103040000220FEF75DFFF7E7000C0020004800407B
:10305000F0B5B3B0002845D04178027841EA0225A6
:10306000C178807841EA0023581E5F283ED85F2D42
:103070003AD8E818602837D8012001AE8DF804004E
:1030800003208DF80500580003248DF80600002267
:103090000CE0A81880B2FDF7F5FC070A611CC9B264
:1030A00037554C1CE4B27054521C92B29A42F0D381
:1030B000214601A8FFF781FD611CC9B23055030A02
:1030C000481CC2B273540C4C208A904200D2024673
:1030D000628201A9E068FDF738FA628A0748E16870
:1030E00003F0DCFA33B0F0BD022100E0032103203D
:1030F000FEF706FFF6E70000000C00200048004045
:10310000F0B5B3B0002845D04178027841EA0225F5
:10311000C178807841EA0023581E5F283ED85F2D91
:103120003AD8E818602837D8012001AE8DF804009D
:1031300004208DF80500580003248DF806000022B5
:103140000CE0A81880B2FDF7A5FC070A611CC9B203
:1031500037554C1CE4B27054521C92B29A42F0D3D0
:10316000214601A8FFF729FD611CC9B23055030AA9
:10317000481CC2B273540C4C208A904200D20246C2
:10318000628201A9E068FDF7E0F9628A0748E16818
:1031900003F084FA33B0F0BD022100E003210420E3
:1031A000FEF7AEFEF6E70000000C002000480040ED
:1031B00010B51E2000F026FDBDE810400320FEF7EC
:1031C0008EBEF8B504464FF4827560684FF4806394
:1031D000A8420AD1A068B0F5004F01D0984204D1AE
:1031E0002068066826F0400606606068A8421ED186
:1031F000A06898420DD00B46009200228021204604
:1032000000F064F808B3606D40F0200060650320B2
:10321000F8BD0B46009200220121204600F056F82E
:1032200098B1606D40F0200060650320F8BD0B464A
:10323000009200220121204600F048F828B1606D7C
:1032400040F0200060650320F8BD0020F8BD0000BC
:103250007CB504460E46154633460122022120461F
:10326000009500F033F828B1606D40F020006065F3
:1032700003207CBD134814490068B0FBF1F04FF403
:103280007A71484301906068B0F5827F0DD1334672
:10329000002280212046009500F018F878B1606D7A
:1032A00040F02000606503207CBD019838B1019892
:1032B000401E019020688068C0430006F5D50020BC
:1032C0007CBD0000A800002000366E012DE9F84307
:1032D00004460F4691461E46089DFDF753FD401BD0
:1032E000351AFDF74FFD804626480068C0F3CB3005
:1032F000684300903AE0701C38D0FDF743FDA0EB26
:103300000800A84203D215B1009858B32BE02068FA
:10331000416821F0E00141606068B0F5827F0BD127
:10332000A068B0F5004F02D0B0F5806F04D12068DE
:10333000016821F040010160A06AB0F5005F09D189
:103340002068016821F4005101602068016841F49F
:103350000051016001205034607000202070032073
:10336000BDE8F88300250098401E00902068806822
:1033700037EA000004D000204845BCD10020EFE728
:103380000120F9E7A800002070470000202109482B
:1033900081611021816108218161C903816120213E
:1033A0000548816110218161082181610805034977
:1033B000886170470010024000040240000C024087
:1033C0002DE9F04F2DED0C8B85B0402000F01AFC5C
:1033D0000120FEF784FD03210020FFF72BFDFE4CAA
:1033E000E07803F0BEFE41EC180B9FEDFCCBB0EE95
:1033F0004C1AF0EE6C1A9FEDFBBBB0EE4B0AF0EEF0
:103400006B0A00F079FEB0EE409AF0EE609AA07878
:1034100003F0A7FE53EC192B03F0F2FE41EC190B5D
:103420009FEDF2DBB0EE4B0AF0EE6B0AB0EE4D1AF8
:10343000F0EE6D1A00F060FEB0EE40AAF0EE60AA69
:10344000607803F08EFE53EC1A2B03F0D9FE53EC98
:10345000192B03F0ADFB53EC182B03F0A9FB03F081
:10346000EBFD0190502000F0CDFB0120FEF737FD71
:1034700003210020FFF7DEFCE07803F072FE41EC50
:10348000180BB0EE4C1AF0EE6C1AB0EE4B0AF0EEE0
:103490006B0A00F031FEB0EE409AF0EE609AA07830
:1034A00003F05FFE53EC192B03F0AAFE41EC190B5D
:1034B000B0EE4D1AF0EE6D1AB0EE4B0AF0EE6B0A5C
:1034C00000F01AFEB0EE40AAF0EE60AA607803F0B9
:1034D00048FE53EC1A2B03F093FE53EC192B03F028
:1034E00067FB53EC182B03F063FB03F0A5FD0546C7
:1034F000B0EE4C1AF0EE6C1AB0EE4B0AF0EE6B0A1E
:1035000000F0FAFDDFF8D092BA4CA9F11009B0EE44
:10351000408A99F80000F0EE608A04EB4000B0F8B1
:10352000400003F01EFE53EC182B03F069FE41EC43
:10353000180B284603F015FE53EC182B04F06CF81A
:1035400003F04AFD82464FF080718A4501DD8A46CC
:1035500003E0A948824500DA82469FEDA81BB0EE41
:103560004B0AF0EE6B0A00F0C7FD99F80000B0EED0
:10357000408A04EB4000F0EE608AB0F850104FF043
:10358000000BA1FB0A020BFB0A224FEAEA7501FBC2
:10359000052103F095FD53EC182B03F0C5FB9FEDBF
:1035A000991B53EC112B03F003FB03F015FD804630
:1035B0009FED96ABB0EE4B0AF0EE6B0AB0EE4A1AF6
:1035C000F0EE6A1A00F098FD99F80000B0EE408A1B
:1035D00004EB4000F0EE608A018EA1FB0A020BFBB7
:1035E0000A2201FB052103F06BFD53EC182B03F0BD
:1035F0009BFB41EC190BB0EE4D1AF0EE6D1AB0EEDC
:103600004B0AF0EE6B0A00F077FD99F80000B0EE7F
:10361000408A04EB4000F0EE608A008A03F0A1FDCE
:1036200053EC182B03F0ECFD53EC192B03F0C0FA0C
:1036300004F0E2F80F460646764A0B21901BB9418A
:1036400002DA16460B2707E07348301A57F10700D5
:1036500002DA714E6FF00707B0EE4B8AF0EE6B8A1C
:10366000B0EE4C1AF0EE6C1AB0EE480AF0EE680AB2
:1036700000F042FDDFF86091B0EE409AA9F1100928
:10368000F0EE609A99F8000004EB4000018C0022F3
:10369000A1FB0A0302FB0A3201FB052103F010FD26
:1036A00053EC192B03F040FB41EC1B0B9FED5BDB54
:1036B000B0EE480AF0EE680AB0EE4D1AF0EE6D1A60
:1036C00000F01AFD99F80000B0EE409AF0EE609A12
:1036D00034F8100003F045FD53EC192B03F090FD76
:1036E00053EC1B2B03F064FA04F086F804460D46F5
:1036F0004C490320091BA84102DA4A4C032507E084
:103700004948201A55F1010002DA474C6FF00105D3
:1037100000BF4FF000099FED45CBB8F5FA6F59DABD
:103720009FED441BB0EE480AF0EE680A00F0E4FC9E
:10373000B0EE40BAF0EE60BA504603F0AAFC41EC9D
:10374000100BB0EE481AF0EE681A00F0D5FC9FEDB1
:103750003B9B51EC100B53EC192B03F051FD53EC38
:103760001B2B03F0E1FA03F037FC83469FED351B7A
:10377000B0EE480AF0EE680A00F0BEFCB0EE40BAC7
:10378000F0EE60BAA8F5FA6003F083FC814641ECE4
:10379000100BB0EE481AF0EE681A049100F0ACFC81
:1037A00053EC192B51EC100B03F02AFD53EC1B2B9F
:1037B00003F0BAFA03F010FC8246B0EE491AF0EEBC
:1037C000691AB0EE480AF0EE680A00F095FCB0EE17
:1037D000409A3BE09AE000006C02002000000000EC
:1037E0000000204000000000000000400000000039
:1037F00000003040200C0020000100FF000000000D
:10380000000037400000000000409F400000000022
:1038100000001C400000F4FFF8FF0F000000000053
:1038200000002E400000FCFFFEFF0300000000002F
:103830000000104000000000008040400000000038
:1038400000000840000000000000F03F0499F0EE86
:10385000609A41EC109BB0EE481AF0EE681A00F046
:103860004BFC9FED751B51EC100B53EC112B03F02F
:10387000C7FC53EC192B03F057FA03F0ADFB81465C
:1038800040F2DC5018EB000F3FDA08F2DC5003F096
:1038900000FCB0EE48BAF0EE68BACDE9021041EC97
:1038A000100BB0EE4B1AF0EE6B1A00F025FC53EC47
:1038B0001A2B51EC100B03F0A3FC41EC190B5046F2
:1038C00003F0E7FB53EC192B03F072F903F084FBD0
:1038D0008246DDE9021041EC100BB0EE4B1AF0EE1F
:1038E0006B1A00F009FC53EC1C2B51EC100B03F08D
:1038F00087FC41EC190B484603F0CBFB53EC192B2A
:1039000003F056F903F068FB814646E09FED4C1B3F
:10391000B0EE480AF0EE680A00F0EEFBB0EE409A16
:10392000F0EE609A504603F0B4FB41EC100BB0EEA1
:10393000481AF0EE681A00F0DFFB53EC1A2B51EC3A
:10394000100B03F05DFC53EC192B03F0EDF903F0C1
:1039500043FB8346B0EE4C1AF0EE6C1AB0EE480A08
:10396000F0EE680A00F0C8FBB0EE409AF0EE609A04
:10397000A8F5FA6003F08DFB41EC100BB0EE481A8D
:10398000F0EE681A00F0B8FB53EC192B51EC100B59
:1039900003F0CAF903F020FB8246A8EB0B00DFF826
:1039A000A880C8F80400B6EB0A0667EBEA77B4EB28
:1039B000090465EBE975B0EE4D1AF0EE6D1AB0EE44
:1039C000480AF0EE680A00F097FBB0EE40AAF0EE6D
:1039D00060AA3046394603F073FB41EC190B9FEDAA
:1039E0001B1BB0EE480AF0EE680A00F085FB019957
:1039F0000022A4FB010305FB013104FB0211B0EE20
:103A0000408AF0EE608A03F05BFB53EC182B03F066
:103A10008BF953EC192B03F0FFFD53EC1A2B03F039
:103A200083F903F0D9FAC8F8080000BF05B0BDEC6F
:103A30000C8BBDE8F08F0000000000000000144077
:103A400000000000008042405C02002000000000F6
:103A500000003540FDF79CB970B52E48016821F093
:103A6000070141F005010160016801F00701052926
:103A7000FAD12949086840F4804008602748026864
:103A800042F4803202600268C2F34042002AFAD057
:103A9000224A234B121D1468224D2C4023431360ED
:103AA000136823F440331360026842F080720260AE
:103AB0000268C2F34062002AFAD04868C0F380303E
:103AC0000028FAD015480830016821F0F0010160A3
:103AD000016821F4E05141F4A0510160016821F432
:103AE000604141F400410160016821F0030141F0AF
:103AF00002010160016801F00C010829FAD10A48AD
:103B0000FDF7F2FF0020FDF765F9002801D0FCF772
:103B1000B6FF70BD003C024000700040003802401B
:103B2000042A40000080BFFF007A030A02480168AF
:103B300041F470010160704788ED00E02DE9F0412B
:103B4000284F3869C0F30000002845D0264E706821
:103B5000401C706000240125042801DD356074607C
:103B6000F068401CF060092801DDB560F460706900
:103B7000401C7061182801DD35617461F069401CDA
:103B8000F061312801DDB561F461306A401C3062BA
:103B9000632806DD34621548006806281ED002F04E
:103BA0001DFBB06A401CB062B0F5967F01DB756208
:103BB000B462306B401C3063B0F5FA7F01DBF56214
:103BC0003463B06B401CB063B0F57A7F01DB756382
:103BD000B4636FF001003861BDE8F08102F03CFB96
:103BE000DFE7000000040040580000202000002013
:103BF00002F06ABD704702F001BA02F009BD02F09E
:103C0000AFBCFEE710B50D490022CA600C31087048
:103C1000FCF7BCFE0A2002F099F8084901231A4675
:103C20000C310748FDF7BCFA18B1FFF7AFFB0120D4
:103C300010BDFFF7ABFB002010BD00005C020020B0
:103C400010030020014A22F810107047780100206C
:103C50002DE9F04FB5B007460020349082467878C1
:103C6000397840EA0129F878B97840EA01283879AA
:103C70003390A8F101004F2860D83398B8EBC00FFB
:103C80005CD8B9F15F0F57D809EB0800602853D80A
:103C90000025002621E0B81990F805B00024012085
:103CA000A04010EA0B0F02D04FF47F4100E000214A
:103CB00009EB050080B200F0ABF86D1CADB24545D4
:103CC00002D34FF0010A03E0641CE4B2082CE6D3EF
:103CD000BAF1010F04D0761CF6B233988642DAD3DB
:103CE0003499012201AC481CC0B262540F22411C1D
:103CF000C9B2225460183A680260091DCDB2294643
:103D000001A8FEF75AFF691CC9B26055030A481C96
:103D1000C2B263540C4C208A904200D202466282A6
:103D200001A9E068FCF711FC628A0848E16802F02A
:103D3000B5FC35B0BDE8F08F022100E003210F2073
:103D4000FEF7DEF8F5E70000000C00200048004018
:103D5000F0B5B3B004460027002C4BD06078217832
:103D600040EA0126E078A17840EA01252079691E21
:103D70005F2943D8B0EB450F40D15F2E3CD8701976
:103D8000602839D800230BE004EB430081794079A7
:103D900041EA0021F01880B2FFF754FF5B1C9BB290
:103DA000AB42F1D3012101AD781CC0B2E95510221C
:103DB000411CC9B22A54681822680260091DCCB29D
:103DC000214601A8FEF7F9FE611CC9B22855030A75
:103DD000481CC2B26B540C4C208A904200D202465E
:103DE000628201A9E068FCF7B0FB628A0748E168DB
:103DF00002F054FC33B0F0BD022000E00320C1B259
:103E00001020FEF77DF8F5E7000C00200048004088
:103E100010B51038C21700EB527323F00702801A56
:103E200001228240074CD810B1F57F4F05D0002900
:103E300002D1215C9143215410BD215C11432154D6
:103E400010BD0000140C002010B5B2B0044660781C
:103E5000217840EA0120E178A27841EA0221002994
:103E600008D0B1F57F4F05D003210520FEF748F8B3
:103E700032B010BD5F2824D8FFF7CAFF01208DF8AB
:103E8000000005208DF801002068CDF80200062111
:103E90006846FEF792FE8DF80600010A08208DF8AC
:103EA0000710094C228A082A00D30246628269461A
:103EB000E068FCF74AFB628A0448E16802F0EEFB26
:103EC000D6E70221D1E70000000C002000480040A6
:103ED00010B5B2B00346002B2CD05878197840EAC0
:103EE0000120D9789A7841EA02215F2824D8FFF787
:103EF000A9FE01208DF8000006218DF80110186838
:103F0000CDF802006846FEF758FE8DF80600010A5B
:103F100008208DF807100B4C228A082A00D302468D
:103F200062826946E068FCF710FB628A0648E16835
:103F300002F0B4FB32B010BD02210620FDF7E0FF15
:103F4000F8E70000000C00200048004004484FF44F
:103F50000031816104218161082181617047000085
:103F6000000802402DE9F0410024194E4FF4802052
:103F7000B0610A2001F0EAFE0420B0610A2001F0DD
:103F8000E5FE01213046FDF765FD012800D1012441
:103F900000254FF400276400B7610A2001F0D6FE27
:103FA0000821B161052001F0D1FE01213046FDF765
:103FB00051FD012801D144F00104052001F0C6FEA5
:103FC0006D1CEDB20F2DE6D3A0B2BDE8F08100006C
:103FD0000008024003B401984100009850EAC12053
:103FE00018BF04204A0D18BF40F0010040F2FF72D4
:103FF000B2EB515F08BF40F00200012808BF052066
:1040000002B07047002809DB00F01F020121914037
:104010004009800000F1E020C0F80011704700283E
:1040200009DB00F01F02012191404009800000F1EE
:10403000E020C0F800117047002809DB00F01F02E3
:10404000012191404009800000F1E020C0F80011FA
:104050007047000002480068C0F30220704700006B
:104060000CED00E002480068C0F302207047000039
:104070000CED00E00907090E002804DB00F1E02048
:1040800080F80014704700F00F0000F1E02080F885
:10409000141D70470907090E002804DB00F1E02019
:1040A00080F80014704700F00F0000F1E02080F865
:1040B000141D70470907090E002804DB00F1E020F9
:1040C00080F80014704700F00F0000F1E02080F845
:1040D000141D70470907090E002804DB00F1E020D9
:1040E00080F80014704700F00F0000F1E02080F825
:1040F000141D7047000000002DE9F04D2DED040B5C
:104100002DED0E8B96B0DDE92550279CDDF890A0B3
:1041100025F0004624F00048BAF1000F14BF012139
:10412000002101EB4502FC4953184A1093422AD35F
:10413000002814BF0123002303EB44030B44F74979
:104140008B4220D358EA00019FEDF59B76D0DFF833
:10415000D8B35D4503D1BAF1000F05D188E0BAF1BB
:10416000000F08BF002100D0012101EB450111F52E
:10417000001F08D8002814BF0121002101EB4401D1
:1041800011F5001F0BD99DED261B9DED240B16B0DC
:10419000BDEC0E8B04B0BDE8F04D00F069BE002709
:1041A000002DBCBFE149884521DAE1498845A8BF17
:1041B00002271CDAC3451ADCDE4901EB2851142919
:1041C00008DDC1F1340220FA02F101FA02F2824262
:1041D0000DD108E058B9C1F1140228FA02F101FA30
:1041E00002F2424503D101F00101C1F1020756EA92
:1041F0000A0124D1002C22DA002D18BF022F01D091
:10420000012F0AD00220FCF714FA16B0BDEC0E8B79
:1042100004B0BDE8F04D00F013BE0220FCF709FA2F
:1042200000F00EFE51EC100B02F0B6FC41EC100B4E
:1042300016B0BDEC0E8B04B0BDE8F08D18E09FED1C
:10424000BEAB9FEDBF8B002871D1B848804522D10D
:1042500005F1804010F5801008BFBAF1000F07D0BB
:10426000B3450ADC002CA8BF9DED260BE0DA0DE07B
:10427000B0EE490AF0EE690ADAE7002C06DA9DEDA5
:10428000260B51EC100B02F087FC6FE0AE4878442F
:1042900090ED000BCCE7D8454DD1002C48DA2EB17B
:1042A00086423AD1BAF1000F42D126E0BAF1000FAE
:1042B00013D00220FCF7BDF900F0F6FD8DED020BE6
:1042C0009DED240B8DED000B10EE900A039961F328
:1042D0001E0003909DED020BAAE78DED02AB9DED54
:1042E000240B1AEE901A10EE900A8DED000B61F37C
:1042F0001E0003909DED020B9AE78DED028B9DED64
:10430000240B18EE901A10EE900A8DED000B61F35D
:104310001E0003909DED020B8AE709DA9DED240B48
:1043200051EC190B53EC102B02F0FEFC1EE020E0C8
:104330009DED240B7CE786421BDAB4F1804F0DD053
:10434000A4F10050B0F1FF5013D1002D11DB9DED11
:10435000240B51EC100B02F08FFA07E09DED240BBB
:1043600053EC102B51EC100B00F0C2BC41EC100BC5
:104370005EE79DED240B51EC100B01F001FDBAF14D
:10438000000FCDE90E0142D19FED710B46B3A6F1AE
:10439000E040B0F17F600CD05E4538D1002D00DAEE
:1043A000A7B3022F0CBF01204FF0FF3002F071FEC7
:1043B000DCE7002D01DD002C0DDA002D01DD002CE5
:1043C0001FDB002D16DA002C14DB012F08BF9FED38
:1043D000620B3FF42DAFB0EE4A0AF0EE6A0A27E70F
:1043E000022F18BF002D0CD0012F0AD1002DFFF68F
:1043F0001FAF06E0002DB8BF002C08DA012F3FF4F4
:1044000017AFB0EE480AF0EE680A11E71BE0012092
:1044100000EBE57050EA070115D0791EB0EE498A2D
:10442000F0EE698A084308BF9FED4D8B4E4800258A
:10443000804570DD4D494E48884514DDB0420DDBA6
:10444000002C19DB2FE00120FCF7F3F816B0BDECCF
:104450000E8B04B0BDE8F04D00F016BDB34502DC94
:10446000002C09DC1FE0864202DA002C1BDA03E094
:104470005E452BDD002C16DD0220FCF7DAF800F09B
:1044800013FD8DED020B53EC1A2B51EC180B02F0BF
:10449000B7FECDE900010399019861F31E00039076
:1044A0009DED020BC4E60220FCF7C3F800F00CFD02
:1044B00010EE901A18EE900A8DED020B8DED008B28
:1044C00061F31E0003909DED020BB1E69DED0E0B16
:1044D00053EC192B51EC100B03F09EF89FED260BBB
:1044E000CDE9080153EC102B9DED080B51EC100B9E
:1044F00002F086FE9FED221B53EC112B02F0B4FF5D
:104500009DED081B53EC112B02F07AFE9FED1E1B54
:1045100053EC112B3CE08CE0FFFF1F00FFFF0F006E
:10452000000000000000F03F0000F03F0000F07FBE
:104530000000404301FCFFFF000000000000F07F8E
:10454000000000000000000026380000000000000D
:104550000000000000000080000000000000F0FFEC
:10456000000000000000F0BF0000E0410000F04348
:10457000FFFFEF3F00000000000000000000D03F00
:10458000555555555555D53F000000000000E03FFA
:1045900002F06AFF9DED080B41EC1A0B53EC102B57
:1045A00051EC100B02F02CFE53EC1A2B02F028FEFB
:1045B00041EC1A0B9FEDFE0B53EC102B9DED080BFD
:1045C00051EC100B02F01CFE41EC1B0B9FEDFA0BA3
:1045D00051EC1A0B53EC102B02F012FE41EC1A0BAB
:1045E0009FEDF70B53EC102B9DED080B51EC100BCE
:1045F00002F006FE53EC1A2B03F00EF841EC1A0BF6
:1046000051EC1B0B53EC1A2B02F0D2FA0690CDE9B9
:1046100006519DED060B53EC1B2B51EC100B02F0D9
:10462000FBFF53EC1A2B02F01FFF41EC100B00F0C4
:10463000A1B90020B6F5801F0EDA9FEDE30B53EC15
:10464000102B9DED0E0B51EC100B02F0D9FDCDE9B6
:104650000E016FF034000E4600EB2650A0F2FF373B
:10466000C6F31300DA4940F07F6646F040568842B0
:10467000D8BF002408DDD7498142C8BF012403DC2C
:104680000024A6F580167F1CD348784400EBC400B4
:104690000F9690ED00CB9DED0E0B53EC1C2B51ECC7
:1046A000100B02F0B9FF9DED0E0B41EC1B0B53EC10
:1046B0001C2B51EC100B02F07BFA41EC100B51EC6F
:1046C000190B53EC102B02F02FFB41EC1D0B51EC9E
:1046D0001B0B53EC1D2B02F093FD41EC1A0BBF4852
:1046E0008DED10AB7844109590ED000B4FF000501D
:1046F00040EA660000EB84408DED080B00F50020D9
:1047000009909DED080B53EC1C2B51EC100B02F0A3
:1047100083FF9DED0E1B53EC112B02F0A5FE41EC27
:10472000100B53EC102B9DED100B51EC100B02F005
:1047300067FD9DED080B41EC1C0B53EC102B9DED20
:10474000100B51EC100B02F05BFD53EC1B2B02F035
:104750008BFE53EC1C2B02F05FFF53EC1D2B02F081
:104760004FFD41EC1C0B53EC1A2B51EC1A0B02F0D1
:1047700047FD41EC1B0B9A480621B0EE4B0AF0EEC8
:104780006B0A784400F0E0FAB0EE401AF0EE601ADE
:10479000B0EE41DAF0EE61DA53EC1B2B51EC1B0B5F
:1047A00002F02EFD53EC1D2B02F02AFD9DED100BA7
:1047B00041EC1B0B53EC1A2B51EC100B02F0F8F9E7
:1047C00053EC1C2B02F01CFD53EC1B2B02F0F0F9F8
:1047D0009DED100B41EC1B0B53EC102B51EC100B0F
:1047E00002F00EFD41EC1D0B9FED7FEB53EC1E2BF9
:1047F00002F0DEF953EC1B2B02F0DAF90890CDE958
:1048000008519DED080B53EC1E2B51EC100B02F0E0
:1048100003FF53EC1D2B02F0FFFE53EC1B2B02F0A9
:1048200023FE9DED080B41EC1D0B53EC102B9DED71
:10483000100B51EC100B02F0E3FC41EC1B0B53ECA2
:104840001A2B51EC1D0B02F0DBFC9DED080B41EC2B
:104850001A0B53EC102B51EC1C0B02F0D1FC53EC57
:104860001A2B02F0A5F941EC1A0B51EC1B0B53EC7F
:104870001A2B02F09DF90C90CDE90C519DED0C0B1B
:1048800053EC1B2B51EC100B02F0C6FE53EC1A2B11
:1048900002F0EAFD41EC1B0B9FED550B53EC102B86
:1048A0009DED0C0B51EC100B02F0AAFC41EC1A0B25
:1048B0009FED510B51EC1B0B53EC102B02F0A0FCA5
:1048C00041EC1B0B9FED4E0B53EC102B9DED0C0B95
:1048D00051EC100B02F094FC53EC1B2B02F068F926
:1048E00041EC100B4848784400EBC40090ED001BED
:1048F00051EC100B53EC112B02F05AF941EC1B0B4D
:10490000384602F0C6FBCDE9080153EC1B2B51ECF5
:104910001A0B02F04DF941EC100B3C48784400EBC7
:10492000C40090ED00CB51EC100B53EC1C2B02F0AB
:104930003FF99DED081B53EC112B02F039F906905D
:10494000CDE906519DED080B53EC102B9DED060BA8
:1049500051EC100B02F060FE53EC1C2B02F05CFEDD
:1049600053EC1A2B02F058FE53EC1B2B02F07CFD8B
:1049700041EC100B9DED261B53EC102B8DED001B15
:1049800000959DED260B51EC100B02F039FC9DEDCE
:10499000000B41EC1A0B53EC102B9DED260B51EC48
:1049A000100B02F039FE9DED061B53EC112B2FE08E
:1049B000000000604715F73FFE822B654715F73F63
:1049C00044DF5DF80BAE543E0000000000004043A1
:1049D0008E9803007AB60B00A2330000D03300009B
:1049E000DA32000000000000000000000000084073
:1049F000000000E009C7EE3FFD033ADC09C7EE3FC7
:104A0000F5015B14E02F3EBE66310000203100004E
:104A100002F0F6FB53EC1A2B02F0CAF89DED060BE0
:104A200041EC1A0B53EC102B9DED000B51EC100BCD
:104A300002F0E6FBCDE90C019DED0C0B51EC1A0BDD
:104A400053EC102B02F0B4F8CDE902010C46AA4950
:104A50008C422FDB611A084318D19DED0C0B53ECEF
:104A6000102B9DED020B51EC100B02F0D5FD41EC2B
:104A70001B0B9FEDA30B51EC1A0B53EC102B02F008
:104A800097F853EC1B2B02F0B9FC2DD20220FBF758
:104A9000D0FD00F009FA10EE901A18EE900A8DED94
:104AA000020B8DED008B61F31E0003909DED020B58
:104AB000FFF7BEBB944A24F00041914214D39349BE
:104AC000214408437FF4EFAC9DED0C0B53EC102B0D
:104AD0009DED020B51EC100B02F09EFD53EC1A2BD6
:104AE00002F08CFC7FF6DFAC24F000408849894A54
:104AF000002601EB205182422BDA481C4FF4801132
:104B000021FA00F02044844AC0F30A517A44A1F209
:104B1000FF3192ED000B814A8DED080BCA4020EA6F
:104B20000202C0F3130040F48010C1F1140120FA16
:104B300001F60992002CB8BF76429DED080B53ECAC
:104B4000102B9DED0C0B51EC100B02F065FDCDE927
:104B50000C019DED0C0B51EC1A0B53EC102B02F0D9
:104B600027F89FED6F0B0890CDE9085153EC102BFF
:104B70009DED080B51EC100B02F042FB41EC1B0BBE
:104B80009FED690B53EC102B9DED080B51EC100BB6
:104B900002F036FB9DED0C0B41EC1C0B53EC102B83
:104BA0009DED080B51EC100B02F036FD53EC1A2B67
:104BB00002F05AFC9FED5E1B53EC112B02F020FB20
:104BC00053EC1C2B01F0F4FF41EC1A0B51EC1B0BC6
:104BD00053EC1A2B01F0ECFFCDE902019DED020B25
:104BE00053EC1B2B51EC100B02F016FD53EC1A2B5F
:104BF00002F03AFC9DED020B41EC1A0B53EC102B2A
:104C000051EC100B02F0FCFACDE908014A489DED89
:104C1000080B0521784400F097F89DED081B51EC36
:104C2000100B53EC112B02F0EBFA9DED021B53EC31
:104C3000112B02F019FCCDE906019DED020B53EC9E
:104C40001A2B51EC100B02F0DBFA53EC1A2B01F08B
:104C5000AFFF9FED3B0B41EC1A0B53EC102B9DED7E
:104C6000060B51EC100B02F0D7FC9DED060B41EC4E
:104C70001B0B53EC102B9DED020B51EC100B02F0B3
:104C8000BFFA53EC1B2B02F04FF853EC1A2B02F037
:104C9000C3FC9DED021B53EC112B02F0BDFC53EC49
:104CA000192B02F0E1FBCDE9020101EB06500115E1
:104CB0000029C8BF039015DC9DED020B324651EC74
:104CC000100B02F02CFEFFF785F9042808BF00F056
:104CD000FBF832469DED020B51EC100B02F01FFE6B
:104CE000CDE902019DED020B51EC180B53EC102B9A
:104CF00002F086FAFFF73ABB000090400000000087
:104D0000FE822B654715973C00CC904000346F3FE6
:104D100001FCFFFF0000E03FA82F0000FFFF0F0095
:104D200000000000432EE63F396CA80C615C20BEF9
:104D3000EF39FAFE422EE63F782E00000000000018
:104D4000000000000000004070B504462DED028B0D
:104D50004D1E00EBC500B0EE408AF0EE608A90ED8B
:104D6000000B35F0060017D053EC182B51EC100B4C
:104D700002F046FA41EC100B6D1E04EBC50090EDFD
:104D8000001B51EC100B53EC112B01F011FF41EC07
:104D9000100B35F00600E7D1022D36D0042D1CD0C3
:104DA000062D1CBFBDEC028B70BD53EC182B51ECD3
:104DB000100B02F025FA94ED0A1B53EC112B01F0B5
:104DC000F7FE53EC182B02F01BFA94ED081B53EC82
:104DD000112B01F0EDFE41EC100B53EC182B51ECB4
:104DE000100B02F00DFA94ED061B53EC112B01F0A1
:104DF000DFFE53EC182B02F003FA94ED040B53EC96
:104E0000102B01F0D5FE41EC100B53EC182B51EC9C
:104E1000100B02F0F5F994ED021B53EC112B01F08D
:104E2000C7FE53EC182B02F0EBF994ED001B53EC8A
:104E3000112B01F0BDFEBDEC028B41EC100B70BDDF
:104E40009FED070B10B553EC102B9FED070B51ECAA
:104E5000100B01F069FF41EC100B10BD00000000C9
:104E60000000000000000000000000000000F03F13
:104E700010B553EC112B51EC100B01F099FE41ECE5
:104E8000100B10BD000000009FED050B10B553EC9A
:104E9000102B51EC100B01F047FF41EC100B10BD33
:104EA00000000000000000009FED050B10B553EC62
:104EB000102B51EC100B02F0A3F941EC100B10BDBC
:104EC00000000000000000709FED050B10B553ECD2
:104ED000102B51EC100B02F093F941EC100B10BDAC
:104EE0000000000000000010014906200870704713
:104EF000E40C002030B5184A1848111D03785B589F
:104F000004786FF30F0343F0030363501449144B09
:104F10004C33114D047808356351124B04782D1D24
:104F200063510378D358047843F0010313512023CD
:104F300093600378D358007843F0100313508868C7
:104F400040F001008860886840F080408860886890
:104F500040F44070886030BD00640240AA790008C7
:104F600000200140500000202DE9F05F2DED068B60
:104F7000FB498A6842F080428A609FEDFA8B44F2D6
:104F800088799FEDFA9ADFEDFA9A42F6E06544F6E9
:104F90002066DFEDF8AA9FEDF8AAF84C40F6CA4863
:104FA00040F6CC4A40F6C84B40F6CB47082822D200
:104FB000DFE800F00484F6F5F4F3F2F10120FBF7EA
:104FC000EBFB53EC182B51EC100B02F019F902F02B
:104FD00033F880B2A080484511D8A0F56850BC389D
:104FE00000EE100AB8EEC00AC0EE090ABCEEE00AF4
:104FF00010EE100AA080BDEC068BBDE8F09FA0F576
:105000008E418939B9420ED8481C00EE100AB8EE1C
:10501000C00AC0EE090ABCEEE00A10EE100A00F564
:105020007A60A080E7E7A0F5A8415539B9420ED8CB
:10503000481C00EE100AB8EEC00AC0EE090ABCEE29
:10504000E00A10EE100A00F5FA50A080D3E7A0F5B0
:10505000C241213941450DD8481C00EE100AB8EE76
:10506000C00AC0EE290ABCEEE00A10EE100A28447D
:10507000A080C0E7A0F5DA41EC3941450ED8481CC4
:1050800000EE100AB8EEC00AC0EE290ABCEEE00A33
:1050900010EE100A00F57A50A080ACE7A0F5F440BD
:1050A000B63800EE100AB8EEC00AC0EE290ABCEE0F
:1050B000E00A10EE100A3044A0809CE70220FBF7C3
:1050C0006BFB53EC182B51EC100B02F099F801F02C
:1050D000B3FF80B2E08048450ED8A0F56850BD38D7
:1050E00000EE100AB8EEC00AC0EE290ABCEEE00AD3
:1050F00010EE100AE0807EE7A0F58E418939414527
:105100000ED8481C00EE100AB8EEC00AC0EE290AFC
:10511000BCEEE00A10EE100A00F57A60E0806AE763
:10512000A0F5A841543941450ED8481C00EE100A9C
:10513000B8EEC00AC0EE290ABCEEE00A10EE100A72
:1051400000F5FA50E08056E7A0F5C2411F3941450D
:105150000DD8481C00EE100AB8EEC00AC0EE290AAD
:10516000BCEEE00A10EE100A2844E08043E7A0F508
:10517000DA41EA39594514D8481C00EE100AB8EE55
:10518000C00AC0EE2A0ABCEEE00A10EE100A00F5D2
:105190007A50E0802FE7A9E22BE2A9E12BE197E02A
:1051A0000FE0A0F5F440B23800EE100AB8EEC00AE5
:1051B000C0EE2A0ABCEEE00A10EE100A3044E0808D
:1051C00019E70320FBF7E8FA53EC182B51EC100B0E
:1051D00002F016F801F030FF80B2E08244F28771ED
:1051E0009FED670A88420ED8A0F56850B83800EEE7
:1051F000900AF8EEE00A80EE801ABCEEC10A10EECA
:10520000100AE082F7E6A0F58E41883940F6CE42DA
:1052100091420ED8481C00EE900AF8EEE00A80EEAB
:10522000801ABCEEC10A10EE100A00F57A60E08226
:10523000E1E6A0F5A841573940F6CD42914210D899
:10524000481C00EE100AB8EEC00ADFED4E0A80EEF0
:10525000201ABCEEC10A10EE100A00F5FA50E082E6
:10526000C9E6A0F5C241253941450DD8481C00EEDC
:10527000900AF8EEE00A80EE801ABCEEC10A10EE49
:10528000100A2844E082B6E6A0F5DA41F039B942C6
:105290000ED8481C00EE100AB8EEC00AC0EE0A0A8A
:1052A000BCEEE00A10EE100A00F57A50E082A2E6A9
:1052B000A0F5F440BB3800EE100AB8EEC00AC0EE0C
:1052C0000A0ABCEEE00A10EE100A3044E08292E6D0
:1052D0000420FBF761FA53EC182B51EC100B01F092
:1052E0008FFF01F0A9FE80B2208344F289718842C9
:1052F0000ED8A0F56850BC3800EE100AB8EEC00A0F
:10530000C0EE0A0ABCEEE00A10EE100A208372E634
:10531000A0F58E418A3951450ED8481C00EE100A7E
:10532000B8EEC00AC0EE0A0ABCEEE00A10EE100A9F
:1053300000F57A6020835EE6A0F5A8415739514513
:1053400022D8481C00EE100AB8EEC00AC0EE0A0AC5
:10535000BCEEE00A10EE100A00F5FA5020834AE68F
:10536000002001400000000000002440FCA9513F43
:105370009A99513FD578513F5EBA513FB80000200D
:1053800023DB513FC1CA513FA0F5C2412439B94284
:105390000DD8481C00EE100AB8EEC00AC0EE090A8B
:1053A000BCEEE00A10EE100A2844208323E6A0F5A4
:1053B000DA41F039B9420ED8481C00EE100AB8EEB6
:1053C000C00AC0EE090ABCEEE00A10EE100A00F5B1
:1053D0007A5020830FE6A0F5F440BB3800EE100AA7
:1053E000B8EEC00AC0EE090ABCEEE00A10EE100AE0
:1053F00030442083FFE50520FBF7CEF953EC182B52
:1054000051EC100B01F0FCFE01F016FE80B260833F
:1054100048450ED8A0F56850BB3800EE100AB8EE2B
:10542000C00AC0EE0A0ABCEEE00A10EE100A608361
:10543000E1E5A0F58E41893951450ED8481C00EEB2
:10544000100AB8EEC00AC0EE0A0ABCEEE00A10EE7E
:10545000100A00F57A606083CDE5A0F5A8415639C1
:1054600051450ED8481C00EE100AB8EEC00AC0EE36
:105470000A0ABCEEE00A10EE100A00F5FA5060834A
:10548000B9E5A0F5C2412339B9420DD8481C00EE58
:10549000100AB8EEC00AC0EE090ABCEEE00A10EE2F
:1054A000100A28446083A6E5A0F5DA41EF394145AA
:1054B0000ED8481C00EE100AB8EEC00AC0EE290A49
:1054C000BCEEE00A10EE100A00F57A50608392E517
:1054D000A0F5F440B93800EE100AB8EEC00AC0EEEC
:1054E000290ABCEEE00A10EE100A3044608382E51F
:1054F0000620FBF751F953EC182B51EC100B01F07F
:105500007FFE01F099FD80B2A08344F2847188424D
:1055100010D8A0F56850BA3800EE100AB8EEC00AEC
:10552000DFEDB10A80EE201ABCEEC10A10EE100ABF
:10553000A08360E5A0F58E41853959450ED8481CF9
:1055400000EE100AB8EEC00AC0EE2A0ABCEEE00A6D
:1055500010EE100A00F57A60A0834CE5A0F5A84192
:105560004E3959450ED8481C00EE100AB8EEC00A54
:10557000C0EE2A0ABCEEE00A10EE100A00F5FA505E
:10558000A08338E5A0F5C241173959450DD8481C0C
:1055900000EE100AB8EEC00AC0EE2A0ABCEEE00A1D
:1055A00010EE100A2844A08325E5A0F5DA41E03981
:1055B00059450ED8481C00EE100AB8EEC00AC0EEDD
:1055C0002A0ABCEEE00A10EE100A00F57A50A08319
:1055D00011E5A0F5F440A83800EE100AB8EEC00AB4
:1055E000C0EE2A0ABCEEE00A10EE100A3044A08396
:1055F00001E50720FBF7D0F853EC182B51EC100B0A
:1056000001F0FEFD01F018FD80B2E08348450ED8A0
:10561000A0F56850BB3800EE100AB8EEC00AC0EE24
:105620000A0ABCEEE00A10EE100AE083E3E4A0F5FB
:105630008E41893951450ED8481C00EE100AB8EE4B
:10564000C00AC0EE0A0ABCEEE00A10EE100A00F52D
:105650007A60E083CFE4A0F5A8415639B9420ED86C
:10566000481C00EE100AB8EEC00AC0EE090ABCEEF3
:10567000E00A10EE100A00F5FA50E083BBE4A0F552
:10568000C2412239B9420DD8481C00EE100AB8EECA
:10569000C00AC0EE090ABCEEE00A10EE100A284467
:1056A000E083A8E4A0F5DA41EE3941450ED8481C64
:1056B00000EE100AB8EEC00AC0EE290ABCEEE00AFD
:1056C00010EE100A00F57A50E08394E4A0F5F4405F
:1056D000B83800EE100AB8EEC00AC0EE290ABCEED7
:1056E000E00A10EE100A3044E08384E40020FBF767
:1056F00053F853EC182B51EC100B01F081FD01F025
:105700009BFC80B2208448450ED8A0F56850BB3879
:1057100000EE100AB8EEC00AC0EE0A0ABCEEE00ABB
:1057200010EE100A208466E4A0F58E418939B94252
:105730000ED8481C00EE100AB8EEC00AC0EE090AE6
:10574000BCEEE00A10EE100A00F57A60208452E404
:10575000A0F5A8415539B9420ED8481C00EE100AF0
:10576000B8EEC00AC0EE090ABCEEE00A10EE100A5C
:1057700000F5FA5020843EE4A0F5C2412139B94237
:105780000DD8481C00EE100AB8EEC00AC0EE090A97
:10579000BCEEE00A10EE100A284420842BE4A0F5A9
:1057A000DA41ED39B9420ED8481C00EE100AB8EEC5
:1057B000C00AC0EE090ABCEEE00A10EE100A00F5BD
:1057C0007A50208417E4A0F5F440B83800EE100AAF
:1057D000B8EEC00AC0EE090ABCEEE00A10EE100AEC
:1057E0003044208407E400003789513FDFED0A0A86
:1057F00020EE200ADFED090A20EE200ADFED080A7C
:1058000080EE201ABCEEC10A10EE100A80B20549E3
:10581000086000F009B800000000C84200008045A0
:1058200000404E45580200202DE9F05F4FF6FF7909
:1058300009EA8000C0F30D054FF40058164EC6F873
:105840001880B714B7610A2000F080FA7804B061BC
:105850000A2000F07BFA00244FF4006A4FF0805BCE
:10586000B761280402D5C6F818A002E04FF0006026
:10587000B0610A2000F06AFAC6F818B00A2000F0F9
:1058800065FA09EA4505641CE4B2102CE8D3C6F8B1
:105890001880BDE8F09F0000000C0240DFED090A0F
:1058A00020EE200ADFED080A20EE200ADFED070ACD
:1058B00080EE201ABCEEC10A10EE100A80B200F091
:1058C00007B800000000C8420000804500404E4577
:1058D0002DE9F05F4FF6FF7B0BEA8000C0F30D056A
:1058E0004FF48077DFF85CA0CAF818704FF40079A5
:1058F000154EC6F818900A2000F028FA4FF080786C
:10590000CAF818800A2000F021FA0024C6F818907E
:10591000280401D5B76101E0C6F818800A2000F01C
:1059200015FA4FF00070B0610A2000F00FFA0BEA90
:105930004505641CE4B2102CE8D3CAF81870BDE821
:10594000F09F0000000002400008024010B504462D
:10595000022221492046FAF7ADFD38B31E49032241
:105960002F392046FAF7A6FD20B31B4903222B3915
:105970002046FAF79FFD08B317490322273920462E
:10598000FAF798FDF0B11449032223392046FAF7BB
:1059900091FDD8B1104903221F392046FAF78AFD3C
:1059A000002817D1BDE8104000F0A6B9BDE81040AE
:1059B00000F038B8BDE8104000F0BAB8BDE81040BB
:1059C00000F018B9BDE8104000F05AB8BDE810402A
:1059D00000F03CB910BD0000217A00080EB50C495A
:1059E0000D2001F13202CDE9002101F117030290EF
:1059F00008A232210A48FAF7C7FC0948FAF73BFD2A
:105A000003B0C1B206485DF804EB00F01FBB000014
:105A1000EF790008257325732573256300000000C6
:105A2000800C00200348012141700278062A00D032
:105A300001707047E40C00200EB50C490D2001F1F7
:105A40000B02CDE9002101F11703029008A23221D7
:105A50000A48FAF799FC0948FAF70DFD03B0C1B2FC
:105A600006485DF804EB00F0F1BA0000EF79000899
:105A7000257325732573256300000000800C00202A
:105A80003EB5002400940194029415480A228168CE
:105A900000780144684600F097FB01216846425CAB
:105AA000303A092A01D8425400E04454491CC9B292
:105AB0000729F4D9401C00F0C1FF9DF800002D28F3
:105AC00001D1B1EE400A07480178062901D005212D
:105AD0000170DFED050A20EE200A80ED010A3EBDCF
:105AE00070020020E40C002000007A440EB50B493F
:105AF0000D20CA1CCDE9002101F11703029008A274
:105B000032210A48FAF740FC0848FAF7B4FC03B01F
:105B1000C1B206485DF804EB00F098BAEF790008CE
:105B2000257325732573256300000000800C002079
:105B30001CB500240094019412490878401CC0B29E
:105B40000870896805220144684600F03DFB0E4953
:105B500068460522491CFAF7ADFC0C4950B18C701F
:105B60000878012805D18878002802D1012000F0AA
:105B70000FF81CBD0120887008780628F0D002209C
:105B80000870EDE7700200200B7A0008E40C00209A
:105B90001FB513490D23CA1D00280BD001AC01F11C
:105BA0001C000BC40092431F0EA232211048FAF7CA
:105BB000EBFB0BE00A4801AC23300BC40092A0F1D0
:105BC0000C0308A232210A48FAF7DEFB0848FAF76C
:105BD00052FC04B0C1B2BDE81040054800F036BA2E
:105BE000EF7900082573257325732573256300005D
:105BF000800C00207047002000F04AB8012000F01F
:105C000047B800000EB50C490D2001F10F02CDE997
:105C1000002101F11703029008A232210A48FAF785
:105C2000B3FB0948FAF727FC03B0C1B206485DF898
:105C300004EB00F00BBA0000EF7900082573257320
:105C40002573256300000000800C00201CB5002493
:105C5000009401940B490878401CC0B20870896810
:105C600005220144684600F0AFFA0749684605225C
:105C7000491CFAF71FFC054908B1CC701CBD012076
:105C8000C8701CBD700200200B7A0008E40C0020D4
:105C90001FB514490D2301F1130200280BD001ACEC
:105CA00001F11C000BC40092431F0FA232211148C6
:105CB000FAF76AFB0BE00B4801AC23300BC40092EF
:105CC000A0F10C0308A232210A48FAF75DFB09484B
:105CD000FAF7D1FB04B0C1B2BDE81040054800F0AE
:105CE000B5B90000EF790008257325732573257376
:105CF00025630000800C0020094801780022022959
:105D000006D003780121032B06D0C27001707047C2
:105D1000C270032101707047C17004210170704787
:105D2000E40C00204FF4005105488161C9038161F2
:105D30008015044988610449400488617047000067
:105D4000000C0240000002400008024000E000BFDA
:105D5000401E411CFBD170470848016A41F0010117
:105D60000162016A41F010010162016841F0010124
:105D7000016047F230514162704700000008004066
:105D800082B0CDE9000121F0004001909DED000BB3
:105D900002B051EC100B70472DE9F0472DED028B4E
:105DA0002B4C207801284ED104F11402294B206994
:105DB000118823F81010E36801EB0308C4F80C8085
:105DC000244B5188143B23F81010A3681944A16098
:105DD000204B9288283B23F8102063681A446260A5
:105DE000401C2061002509282CDD25610A26B2FB14
:105DF000F6F0194F38806560B1FBF6F040F6E441EB
:105E0000DFF85890484309EB103001F0AAF99FEDF4
:105E1000148B53EC182B00F087FF01F00DF97880FC
:105E2000A560B8FBF6F040F6E441484309EB1030BA
:105E300001F097F953EC182B00F076FF01F0FCF815
:105E4000B882E5602570BDEC028BBDE8F0870000EC
:105E50003C000020FC020020B800002024FAFFFFD4
:105E6000CBA145B6F3FDB43FF0B53C4D3C493D4AAE
:105E700028784FF0010406064FF0000303D5E6052D
:105E80008E61D37102E080268E61D47147064FF493
:105E9000807603D536048E61937101E08E61947132
:105EA00087064FF4007603D536048E61537101E006
:105EB0008E615471C7064FF4806603D536048E6137
:105EC000137101E08E61147107074FF4006603D56A
:105ED00036048E61D37001E08E61D47047074FF4B1
:105EE000805603D536048E61937001E08E61947004
:105EF00087074FF4005603D536048E61537001E0D6
:105F00008E615470C6074FF4804003D0000488614E
:105F1000137001E0886114706878C10704D01249D9
:105F20000B6000F0FE0068706878810705D50F49A6
:105F300002220A7000F0FD0068706878410706D5FB
:105F400047F230510A4A516200F0FB0068706878ED
:105F5000010702D500F0F7006870F0BD140C0020B6
:105F6000001002405002002020000020E40C00201D
:105F70000008004038B5002100910E4CA0600421BB
:105F800021700D49497800290BD0011D0322684674
:105F900000F01AF92078C01C20706846FFF7D6FC84
:105FA00038BD011D0222684600F00EF92078801CE1
:105FB0002070F2E770020020E40C00200849002263
:105FC0000A7088600748C860074808610748486148
:105FD000074888610748C8610748086270470000A1
:105FE000E40C0020DD590008ED5A0008915B000820
:105FF000395A0008055C0008915C0008F8B5104D9E
:106000002868C0F3001000260E4C002808D028682D
:1060100000906868009021790B48FFF7ABFF66603D
:106020002868C0F34010002809D06068322800DDDD
:1060300066606968044A60681154401C6060F8BD7D
:106040000044004070020020B20C00200A460249C1
:106050008B68014601481847E40C002000440040CA
:1060600070B5264C20780025062828D0244E3068AC
:10607000012823D1207878B1207801280FD020780A
:1060800002280FD0207803280FD0207804280FD0C2
:10609000207805280FD010E0FFF7A0FC0DE0FFF7F7
:1060A00025FD0AE0FFF7A7FD07E0FFF7A7FD04E0E5
:1060B000FFF7C2FC01E0FEF717FF356070BD114E1F
:1060C00030680128FAD1A069804794ED010A0E4991
:1060D000B5EEC00AF1EE10FA05DBBCEEC00A10EE18
:1060E000100A088107E0B1EE400ABDEEC00A10EECA
:1060F000100A40420881356070BD0000E40C0020A9
:106100007000002060000020B80000202A4C00260B
:106110002670FAF745FEFDF79FFCFCF75BF8FCF7ED
:106120000DF8FCF7E5F9FCF7BDFAFCF7D7FBFBF738
:106130003DFFFCF773F9FCF769FCFCF78BF9FCF702
:10614000E9FAFCF741FBFCF737FAFCF7F7F91B48D3
:10615000016841F001010160C16841F00101C160C5
:10616000416C41F400414164154D28680128FCD17F
:10617000207840B1012811D0022813D00328F4D18F
:1061800000F0CCFBF1E70F494FF480008861FDF788
:10619000FDF82E602078401C2070E6E70220207079
:1061A0002E60E2E700F0A0FB4020A0612E60207886
:1061B000401C2070D9E700000000002000040040CF
:1061C0008C0000200010024003E011F8013B00F8B1
:1061D000013B521E92B2F8D27047000010B51D4C20
:1061E000206806280CD2DFE800F0030C151E2831C9
:1061F00000220421012000F0B5FC2068401C206032
:1062000010BD00220521012000F0ACFC2068401CDC
:10621000206010BD00220621012000F0A3FC2068B0
:10622000401C206010BD4AF65522FF21022000F0DC
:1062300099FC2068401C206010BD0122F221022040
:1062400000F090FC2068401C206010BD06202060FB
:1062500010BD00002000002070B52DED108BAD4D5D
:106260009FEDADBB9FEDAECB9FEDAFEB9FEDB0FBD8
:10627000B14E9FEDB2DB9FEDB3AB286801280AD089
:106280009FEDB29B02287CD0032801D10120286019
:10629000BDEC108B70BD00F0E5FAAE4C207A00F03A
:1062A00060FF41EC180BB0EE4B1AF0EE6B1AB0EE3B
:1062B0004C0AF0EE6C0AFDF71FFFB0EE409AF0EECC
:1062C000609AE07900F04DFF53EC192B00F098FF35
:1062D00053EC182B00F06CFC53EC1A2B00F024FD4F
:1062E00041EC180BA07900F03CFF41EC190BB0EE2B
:1062F0004B1AF0EE6B1AB0EE4C0AF0EE6C0AFDF79A
:10630000FBFEB0EE40AAF0EE60AA607900F029FF33
:1063100053EC1A2B00F074FF41EC1A0BB0EE4E1A3E
:10632000F0EE6E1AB0EE4C0AF0EE6C0AFDF7E4FEE9
:10633000B0EE40BAF0EE60BA207900F012FF53ECF4
:106340001B2B00F05DFF41EC1B0BB0EE4F1AF0EE83
:106350006F1AB0EE4C0AF0EE6C0AFDF7CDFEB0EE0F
:1063600040CAF0EE60CAE07800F0FBFE53EC1C2B54
:1063700000F046FF53EC1B2B00F01AFC53EC1A2BD9
:1063800000E027E000F014FC53EC192B00F010FCA7
:1063900053EC182B00F00CFC41EC100B85ED020BBC
:1063A00053EC1D2B51EC100B01F028F801D285EDB8
:1063B00002DB9FED690B53EC102B95ED020B51ECBA
:1063C000100B00F01DFF00F037FE70812868401CA4
:1063D00028605DE700F04BFA5E4C2434207A00F030
:1063E000C0FEB0EE4BDAF0EE6BDA41EC180BB0EE1B
:1063F0004D1AF0EE6D1AB0EE4C0AF0EE6C0AFDF795
:106400007BFEB0EE40BAF0EE60BAE07900F0A9FE93
:1064100053EC1B2B00F0F4FE53EC182B00F0C8FBE0
:1064200053EC1A2B00F080FC41EC180BA07900F023
:1064300098FE41EC1B0BB0EE4D1AF0EE6D1AB0EE6B
:106440004C0AF0EE6C0AFDF757FEB0EE40DAF0EEC3
:1064500060DA607900F085FE53EC1D2B00F0D0FE71
:1064600041EC1D0BB0EE4E1AF0EE6E1AB0EE4C0A77
:10647000F0EE6C0AFDF740FEB0EE40EAF0EE60EAA6
:10648000207900F06EFE53EC1E2B00F0B9FE41ECBB
:106490001E0BB0EE4F1AF0EE6F1AB0EE4C0AF0EE93
:1064A0006C0AFDF729FEB0EE40CAF0EE60CAE07853
:1064B00000F057FE53EC1C2B00F0A2FE53EC1E2BF9
:1064C00000F076FB53EC1D2B00F072FB53EC1B2B02
:1064D00000F06EFB53EC182B00F06AFB41EC100B44
:1064E00085ED040B53EC192B51EC100B00F086FFDB
:1064F00001D285ED049B95ED040B53EC1A2B51EC66
:10650000100B00F07DFE00F097FDB0812868401C64
:106510002860BDE68002002000000000000020404E
:1065200000000000000000400000000000003040BB
:106530000000000000003840B8000020000000000B
:10654000007884400000000000408F400000000000
:10655000004050401C0D0020000000000000594089
:10656000F8B5274C2068C0F30010264D0026264BB6
:10657000002835D0206800906068009000202946EF
:106580002A784978012A01D1032902D0022A0AD0A7
:106590000BE059681D4A491C02E02F5C1754401C4F
:1065A0008842FADB1BE0032902D0032A0BD016E055
:1065B000164A59682432491C02E02F5C1754401CCB
:1065C0008842FADB0BE0032909D1104A59684832A6
:1065D000491C02E02F5C1754401C8842FADB5E60C5
:1065E0002068C0F34010002808D05868322800DD29
:1065F0005E60616858682954401C5860F8BD00000E
:1066000000140140C00B0020800200201C0D00205F
:1066100010B51248007803280DD3114B40F2FF3417
:10662000194698880F4A0968A04205D3002098802F
:106630000860EE20506010BD52680B4C2270441C64
:106640009C800A540948016821F001010160002181
:106650004162016841F00101016010BD00000020AD
:10666000000C00200048004094000020001400406E
:10667000084901F50460016000218180C180017238
:10668000A0F58862C2604FF48062028241820248B3
:10669000FBF75BBBC00300200048004070B5084D0D
:1066A000084B074CDB780C34195103212846FBF7C3
:1066B0007FF82846BDE870400321FBF765B800006D
:1066C00000600240CF79000870B509486FF0010101
:1066D0000161016821F001010160064CA088E080A1
:1066E0000025A58001202072FCF7D2FA257270BD2A
:1066F00000140040000C00200448C16841F0010172
:10670000C160016841F00101016070470014004060
:106710002DE9F041FCF754FE3A4D3B4C0A2629780E
:106720000023042925D2DFE801F024022649A868C5
:10673000374A90FBF6FC354F106827F810C0401C14
:106740001060092800DD13600020324A37F810C0BD
:10675000D2F80080C444C2F800C0401C0A28F5DB0F
:106760001068B0FBF6F08E1D24F816001360491C6B
:106770002970BDE8F081A868284A90FBF6FC264FF6
:10678000106827F810C0401C1060092800DD136055
:106790000020234A37F810C0D2F80080C444C2F861
:1067A00000C0401C0A28F5DB1068B0FBF6F08E1D17
:1067B00024F816001360491C2970DAE7A8681A4A01
:1067C00090FBF6FC174F106827F810C0401C1060B3
:1067D000092800DD13600020144A37F810C0D2F8F1
:1067E0000080C444C2F800C0401C0A28F5DB1068D1
:1067F000891DB0FBF6F024F8110013600120287009
:10680000B7E700005C020020B800002098020020DA
:106810003000002024000020AC02002034000020C2
:1068200028000020C0020020380000202C0000209A
:1068300010B50B4C207003206070080AA070E17046
:10684000100A2071062162712046FCF7B6F9A0718A
:10685000000A0821E0712046BDE8104000F06CB944
:10686000080D0020032204210120FFF7E1BF0322CD
:106870003C210220FFF7DCBF00B52DED048B83B077
:1068800041EC190B00F0FCFD41EC180B18EE100A5E
:1068900018EE901A8DED008B002818BF01200843D8
:1068A00020F00040C0F17F6000F1E040C00F14D044
:1068B00019EE101A19EE900A8DED009B002918BFF1
:1068C0000121084320F00040C0F17F6000F1E0406A
:1068D000C00F04BF0120F9F7ACFE51EC180B03B058
:1068E000BDEC048B00BD000010B5FBF735FBFAF7DB
:1068F0002FF8FDF72BFBFFF715FAFFF7FDFEFFF76B
:10690000B7FEFEF7F7FA0448FFF758FBFFF7ACFABB
:10691000BDE81040FFF720BA0D6B000870B52DEDF3
:10692000028BFFF7A1FA3E4C9FED3E8A3E4D208838
:10693000F3EE098A00EE100A3C4EF8EE400A80EEB3
:10694000880AD5ED040AB4EE600AF1EE10FA13D00D
:1069500000EE100AF8EE400A80EE880A85ED040A7F
:1069600010EE100AB04201DDC5ED048AFFF7DAF936
:1069700095ED040AFEF73AFF608800EE100AB8EEC3
:10698000400AC0EE080A95ED050AF4EE400AF1EE61
:1069900010FA13D000EE100AF8EE400A80EE880AD2
:1069A00085ED050A10EE100AB04201DDC5ED058A3D
:1069B000FFF7B8F995ED050AFEF770FF287AFEF7A4
:1069C000D3FAA868401CA860072801DD0020A86051
:1069D000FFF79EFEFFF744FBFFF7DEF9144E307819
:1069E00000F00400E860FDF7BDFA6880C1437170F3
:1069F0006FEA10203070E96800F00400884208D087
:106A0000A088401C80B2A0804FF6DC71884200D97B
:106A1000A1800848406A08490885BDEC028B70BD1A
:106A20007801002000007A44000000200000C841E6
:106A3000AC00002000080040B80000200178174A90
:106A400040F635435143427812FB03F201EB421109
:106A5000827840F2712312FB03F201EB0212C1783B
:106A600001EB4103C3EBC11102EBC102017901EB60
:106A7000C10303EB011102EB81024179807901EB43
:106A8000810102EB4101084400EE100A9FED041A57
:106A9000F8EEC00A80EE810A7047000040420F0005
:106AA0000050C34730B5164800F10C0151E8002FE3
:106AB00042F0100241E80023002BF7D11049114D9C
:106AC000091D114C0F4BA2790833D15000F114016C
:106AD00051E8002F42F0800241E80023002BF7D15B
:106AE000A1796958A27941F01001A9500C3050E801
:106AF000001F41F0200140E80012002AF7D130BD0C
:106B00000044004000600240197A000870B5084D4A
:106B1000084B074C9B790C34195106212846FAF78B
:106B200047FE2846BDE870400621FAF72DBE00005A
:106B300000600240CF79000870B5084D084B074C43
:106B40009B790C3418510A4606212846FAF730FE84
:106B50002846BDE870400621FAF716BE00640240E0
:106B6000CF79000810B50B4C2070062060700B0A1E
:106B7000A370E170110A2171627101462046FCF791
:106B80001CF8A071000A0821E0712046BDE8104001
:106B9000FFF7D2BF080D002081F00041704780F060
:106BA0000040704721F00041704720F000407047DE
:106BB00010B591EA030F48BF83F0004300F134851C
:106BC000841A71EB030C05D2121943EB0C03001B62
:106BD00061EB0C01DFF824E14FEA1154A4EB135CE4
:106BE0001EEA430F18BF9EEA445F73D023EA0E03E8
:106BF000DCF1200E21EA045143F4801332D322FA4F
:106C00000CFE10EB0E0023FA0CFE41EB0E01CCF152
:106C1000200E03FA0EFE10EB0E0051F10001B1F54B
:106C2000801FCCF1200E32D201EB045112FA0EF289
:106C3000BDE8104058BF7047401C38BF5FEA4202B1
:106C400018BF7047002814BF20F0010041F1000177
:106C50004FEA410313F5001F38BF7047A1F1C0414F
:106C600000F0C6BB012A43EB0302ACF1200CDCF1BF
:106C70001F0E32BF4FF0000E23FA0CF310EB03008F
:106C800041EB0451B4EB115FD0D0A1EB045101F5FD
:106C9000801149085FEA300001EB04510ED350F136
:106CA000000038BF12FA0EFE08D1BDE81040C9E757
:106CB000401C38BF5FEA4202CAD1C3E7BDE81040BA
:106CC0004FEA410313F5001F38BF7047A1F1C041DF
:106CD00000F08EBB9EEA445F08D011EA5E0FBDE86B
:106CE000104004BF01F0004100207047BDE8104093
:106CF00070B500F02FFB00BF64FBBE3E0000E0FF5C
:106D000002494FF0000000F0D8BD00BF0000F87F3E
:106D1000491058BFC1F140415B1058BFC3F1404317
:106D20008B42EFF3008070472DE9C04130B4DFF8AB
:106D3000A0C23CEA111418BF3CEA131400F0EC8026
:106D400081EA03051CEA111444EAD57418BF1CEA51
:106D5000131500F0C780A4EB05044FF0004545EA89
:106D6000C12145EAC32341EA505143EA525304F199
:106D70007F74994204F500344FEAC0204FEAC222E2
:106D800008BF904200F09C804FEA13650FF2401656
:106D9000765D4FEA134506FB05F7C7F1807706FBE2
:106DA00007F74FEAD737A7FB03687642C8F5803864
:106DB000A7FB06CE38BFA8F1010807FB08E64FF095
:106DC000000EA6FB028CE6FB03CEDCF1000CCEF13C
:106DD000004E38BFAEF1010EA6FB0C584FF0000775
:106DE0004FF00005E6FB0E87A1FB08C6A0FB07CE0F
:106DF00016EB0E0645F10005E1FB076515F1E04EC7
:106E00007EBFA4F580345FEA46066D4116F1800727
:106E100045F100054FEA17274FEA066647EA05677E
:106E2000A6F1DE46B6F1805F4FEA15251FD9384638
:106E300024F0010C05EBC471BCF1FE6F01EB0C11E9
:106E400002D8F0BCBDE8008124425CBF01F5801E81
:106E50009EEAC47F02D4F0BCBDE80081244238D44D
:106E6000F0BCA1F1C041BDE8004100F0C1BA4FEA59
:106E7000D22242EA43524FEAD323A7FB02864FEACB
:106E8000D02040EA415007FB03661EEA0E0F4FEA8E
:106E9000D12105FB026658BFA6EB0056B6EB0056A3
:106EA0004FEA520E4EEAC37E18EB0E0E56EB530E0F
:106EB000BDD518EB02085E417F1C55F10005B6E711
:106EC0004FF480154FF000074FF000064FF0000818
:106ED000ADE7F0BC4FF0000001F1C04101F000410E
:106EE000BDE8008111EA0C1F0CEA131500D00CE07C
:106EF00013EA0C1F00F025804FF00000F0BC81EA7F
:106F0000030101F00041BDE80081F0BCBDE8004193
:106F100081EA030100F06CBAF0BCBDE8004170B535
:106F200000F018FA097EFC3E00F007B881EA030180
:106F30004FF0000001F00041704781EA030100F0CA
:106F400057BAF0BCBDE800414FF00000214970473E
:106F5000FFFDFBF9F7F5F4F2F0EEEDEBE9E8E6E41E
:106F6000E3E1E0DEDDDBDAD8D7D5D4D3D1D0CFCDA5
:106F7000CCCBCAC8C7C6C5C4C2C1C0BFBEBDBCBBDE
:106F8000BAB9B8B7B6B5B4B3B2B1B0AFAEADACABD9
:106F9000AAA9A8A8A7A6A5A4A3A3A2A1A09F9F9EB3
:106FA0009D9C9C9B9A999998979796959594939365
:106FB000929191908F8F8E8E8D8C8C8B8B8A8989FC
:106FC000888887878685858484838382828181807F
:106FD0000000FF070000F87F4FEA41034FEA5353D8
:106FE000A3F58063D3F11E03C8BFD3F1210C0CDDE0
:106FF0004FF0004242EAC12242EA505232FA03FC08
:107000008CEAE17CACEBE1707047102BC4BF002030
:10701000704703F5787CBCF1FF3F04D06FF000426D
:1070200082EA2100704770B500F094F949922480FB
:1070300000207047F2E700004FEA1153A3F5806388
:10704000D3F11E03A8BFD3F1200C08DB4FF00042A0
:1070500042EAC12252EA505232FA03F07047094222
:107060000BD4102BC4BF0020704703F5787CBCF113
:10707000FF3F05D04FF0FF3070474FF000007047E2
:1070800070B500F067F900BF499224800020704776
:10709000F0E710F0004248BF4042B0FA80F310FA27
:1070A00003F10AD0C3F11D0303F580634FEA415099
:1070B00002EB035202EBD12170474FF00000704702
:1070C0007FEAE17202D1101A62EB0101B1FA81F399
:1070D0000B3B24D3994012D1B0FA80F310FA03F19C
:1070E00008BF7047C3F11D0303F5406303EBC223E0
:1070F0004FEAD1224FEA415002EB03517047C3F1EE
:10710000200C20FA0CFC9840C3F1320303F54063D5
:1071100003EBC22341EA0C0101EB0351704710B5A8
:10712000C3F1320CC3F10004C4F1200E0CF5406C25
:107130000CEBC22201FA0EFC21FA04F100FA0EF364
:10714000E040BDE8104040EA0C0001EB025138BFBE
:107150007047401C41F100015B0008BF20F00100B6
:107160007047B0FA80F310FA03F10AD0C3F11D039F
:1071700003F580634FEA41504FEA035202EBD121FD
:1071800070474FF00000704751EA030C17D41CF50C
:10719000801F58BFBCF5801F00F10680994218BFC0
:1071A000704708BF9042704707D711F5801F58BF3E
:1071B00013F5801F19D499427047894270471CF516
:1071C000801F08D5BCF5801FF7D58B4218BF7047CC
:1071D00008BF824270474FF4001C1CEB410F38BFC0
:1071E0001CEB430F01D28B42704770B500F0B2F830
:1071F000922449004FF000514FF08053FFF788BDB3
:10720000DFF848C170B51CEA111E1EBF1CEA131539
:107210009EEA0C0F95EA0C0F00F06F8081EA0304E0
:1072200023EA4C134EEAD47E21EA4C1141F480113A
:1072300043F48013AE44A1FB024CA0FB0365AEF106
:107240007F7E361955EB0C05A1FB034C4CF1000376
:10725000A0FB021C16EB0C06654153F1000309422A
:1072600018BF46F0010613F4007F0BD14FEA03313B
:107270004FEA0530340341EA155140EA16506FF0E9
:1072800003020AE04FEAC3214FEAC520F40241EAB3
:10729000555140EA56506FF0020202EB2E4201EBCC
:1072A000025585EACE710AD05FEA440C18BF24F07B
:1072B000004450F1000041F1000120EAD47040F296
:1072C000FE7C624500D270BDA84214BF4FF08044DE
:1072D0004FF04044002E08BF0024BEF1806FA8BFCD
:1072E000A1F1C041BDE8704080F282804FF0000003
:1072F00001F1C04101F0004170479EEA0C0F0CEA19
:10730000131518BF95EA0C0F06D04FF0000081EA64
:10731000030E0EF0004170BD00F01CF88900013E24
:1073200000F007B800F009B84FEA430C5FEA5C5C74
:1073300008D081EA030100F05BB84FEA410C5FEA34
:107340005C5CF6D14FF00000014970470000FF0778
:107350000000F87F0EF1020E2EF0030E5EF8046BB3
:10736000364205D4012A43EB030515F5001F12D858
:10737000012841EB010C1CF5001F0CD80ED14FEA7F
:10738000D17C15F5001F0CEB4C0C0CF1020C08BF66
:107390004CEBD37C04E04FF0080C01E04FEAD37CC7
:1073A0000CEB4C0526FA05F606F00706B6F1040CC0
:1073B00006D20EEB860CBDE870404CF0010C604725
:1073C000DFE80CF0090B02024FF000414FF0000023
:1073D000A1F5002170BD19461046012851EB0104AA
:1073E00018BFD4F5001484BF002001F0004170BD27
:1073F0000808A0F500114FEA3101704753EA010C6B
:1074000017D41CF5801F58BFBCF5801F00F1068003
:107410008B4218BF704708BF8242704707D713F5E9
:10742000801F58BF11F5801F19D48B4270479B42B3
:1074300070471CF5801F08D5BCF5801FF7D5994211
:1074400018BF704708BF904270474FF4001C1CEBF8
:10745000430F38BF1CEB410F01D2994270470FB464
:107460000CBC03BCFFF7C1BE91EA030F10B581F05D
:1074700000413FF5A5AB83F0004300F0D5B8000014
:107480002DE9F04101F5801CBCF5001FC0F2A98078
:107490004FEA115C21EA0C510CF1FD0C41F4801112
:1074A0005FEA5C0C0CF5C07C01D34000494130A47C
:1074B000890241EA905187028E0E0A0CA45D04FBFA
:1074C00004F602FB06F6C6F14046A4FB0662F60D82
:1074D00046EA422606FB06F4A4FB01235242C3F10E
:1074E000404338BF5B1EA6FB02420024E6FB032498
:1074F000D20B42EA4446A6FB0623A1FB02E2A3FB11
:1075000007E4E3FB61426442C2F1404E38BFAEF192
:10751000010EA6FB04234FF00002E6FB0E32A2FB95
:1075200003463400E2FB6264A1FB06E6A4FB07E825
:10753000E4FB61687642C8F1405838BFA8F1010801
:10754000A2FB06E4A3FB08E5E2FB6854A1FB05E609
:10755000A7FB04E8E1FB648618F1200556F100065C
:10756000A809A8F11B08B10908F03F08B8F10A0FF3
:1075700040EA86601CD901EB0C51BDE8F08100BFE8
:10758000FCF5EEE8E2DDD8D3CFCBC7C3C0BDB9B6BA
:10759000B4B1AEACA9A7A5A3A19F9D9B9A989695BF
:1075A0009392908F8D8C8B89888786858483828146
:1075B000A0FB006800FB01F208EB4208B8EB87284B
:1075C00007D5341858EB0104D5D5401C51F1000102
:1075D000D1E7341A78EB0104CDD4401E71F10001DB
:1075E000C9E75FEA4C0C5FEA9C5C0DD105D34FF014
:1075F000000001F00041BDE8F081BDE8F04170B548
:10760000FFF7A8FE6DDBFFBEBDE8F0414FF00000C4
:10761000004970470000F87F10B591EA030F48BF9A
:1076200083F000433FF5CCAA841A71EB030C07D218
:1076300012198CF0004C43EB0C03001B61EB0C01A6
:10764000DFF8A4E14FEA1154A4EB135C1EEA430FE8
:1076500018BF9EEA445F00F0B08023EA6E035242F6
:1076600021EA0451C3EB6E0338BF5B1EDCF1200E30
:1076700025D322FA0CFE10EB0E0043FA0CFE41EB70
:107680000E01CCF1200E03FA0EFE10EB0E0051F1AC
:107690000001CCF1200E29D412FA0EF201EB0451B4
:1076A000BDE8104058BF7047401C1CBFB2F1004FEE
:1076B000704700280CBF491C20F00100704712EBF6
:1076C000020E43EB030218BF4FF0010E4EEA4202D6
:1076D000ACF1200CDCF11E0E54D943FA0CFE10EB79
:1076E0000E0051F1FF31CCF11E0ED5D50EF1010E79
:1076F00012FA0EFE404141EB010101EB445C5FEAEE
:107700005C5C10D910EBDE7001EB045138BFBEF1A8
:10771000004FBDE8104018BF704700280CBF491C3F
:1077200020F00100704730D24FEAD42C11F500113F
:1077300024F400641BD0B1FA81F20B3AA41AA41EFF
:10774000D2F12003914030FA03F31943904001EB4A
:10775000CC71002C01EB0451BDE81040A8BF70476C
:1077600001F1C0414FF0000001F000417047B0FA54
:1077700080F310FA03F100D110BDE41A173C48055C
:10778000C90AE4E701EB045110BD491001EB0451B3
:10779000BDE810404FEA300002E04FF000017047B2
:1077A0004A0008BF0042F8D0B2F5001F28BF70475A
:1077B00001F000414FF0000070479EEA445F07D09F
:1077C00011EA5E0FBDE8104004BF002100207047A1
:1077D000BDE8104070B5FFF7BDFD00BF40DFF63ECD
:1077E00083F00041104670470000E0FF4FF040700A
:1077F000E1EE100A704700004FEAC1230A1543EA80
:1078000050534FEAC02C18BF43F000431BD4A2F2E0
:107810004E02D2F57C7240F34280502AA8BF50221B
:1078200023FA02F12CFA02F0D2F1200260B403FA3A
:1078300002F588BF2843C2F1000223FA02F598BF7F
:10784000284360BC704702F57C7212F5826F08BF56
:1078500023F00043D2F12E0221DB1AD0502AA8BF18
:10786000502223FA02F12CFA02F0D2F1200260B485
:1078700003FA02F588BF2843C2F1000223FA02F599
:1078800098BF284360BC4042C1F1000138BF491E87
:1078900070479CF0000F08BF93F0004FDED070B52A
:1078A000FFF758FD9224498000214FF000007047F7
:1078B0006FEAE17080F0004170470CF00F03092B74
:1078C00008BF082000F059800A2B0BD0082B18BFE6
:1078D000704708BF1CF0400F0AD04FF000004FF077
:1078E000000170471CF0400F18BF4FF00040704778
:1078F0001CF0100F08D020F0704300F07F4242EAE5
:10790000D3014FEA4370704700F0604021F07F429E
:1079100042EA000201F07F4040EA727070474FF087
:10792000FF0C4CF4E06C1CEA11531CBF9CEA030CE6
:107930009445C2BFDA4201EB02517047002B0DD0D3
:10794000BCF1000F0FD0002A01F00041A4BF41F0AC
:10795000E04141F07F614FF00000704701F00041CD
:107960004FF00000704750EA01334FF09B0C18BFF6
:107970004CF0806C7FF4C4A970471CF4801F11D0B8
:107980001CF4E02F03D06FEACC31490070474FF070
:107990004050EFF3008222F0704242EA000282F38C
:1079A000008870474FF000007047102840587088DA
:1079B000A0B8000000000404040000080000000853
:1079C00000020406080A0C102840587088A0B8105D
:1079D0002840587088A0B800000000000000000196
:1079E0000203040607080900000000010203042A3C
:1079F0002A00524C5200574C5200524D4400525AE9
:107A00005300575A530025303123002B303030308B
:107A100031002B303030303000102840587088A0B2
:107A2000B85743535230333030310000000000006B
:107A3000000000000000F03F000000000000F83FE0
:107A400000000000000000000000004003B8E23F1A
:107A5000000000000000000006D0CF43EBFD4C3ECC
:107A6000033333333333E33FFFAB6FDBB66DDB3FC1
:107A70004D268F515555D53F01411DA96074D13F09
:107A800065DBC9934A86CD3FEF4E454A287ECA3F03
:107A90003E5555555555C53F93BDBE166CC166BF85
:107AA0002CDE25AF6A56113FF16BD2C541BDBBBE7E
:107AB000D0A4BE726937663E0000000000000000DE
:107AC000E07A00080000002098020000C4010008CD
:107AD000007B0008980200205011000000020008FE
:107AE00001190383FFFF42019210C524F400AA0587
:107AF000C355AAAA5502DE010224010218010000A2
:040000050800018965
:00000001FF
